S01A00004652444D2D4B4C32355A5F4A6F79737469636B2E68657815
S1130000003000208D860000616800006D680000EB
S11300106D6800006D6800006D6800006D68000088
S11300206D6800006D6800006D680000651F0000C9
S11300306D6800006D6800008D1F00002D1F00001A
S11300406D6800006D6800006D6800006D68000058
S11300506D6800006D6800006D6800006D68000048
S11300606D6800006D680000653100006D68000077
S11300703D7F00006D6800006D680000A17B0000FA
S11300806D6800006D6800006D6800006D68000018
S11300906D6800006D6800006D6800006D68000008
S11300A06D6800006D6800006D6800006D680000F8
S11300B06D6800006D6800006D6800006D680000E8
S1130400FFFFFFFFFFFFFFFFFFFFFFFF7EFBFFFF7D
S1130410002934D00123002210B488422CD30124B3
S11304202407A14204D2814202D209011B01F8E748
S1130430E400A14204D2814202D249005B00F8E701
S1130440884201D3401A1A434C08A04202D3001B2D
S11304505C0822438C08A04202D3001B9C08224360
S1130460CC08A04202D3001BDC082243002803D09E
S11304701B0901D00909E3E7101C10BC70470028D0
S113048001D00020C04307B4024802A140180290E2
S113049003BDC046D90000000029F0D003B5FFF722
S11304A0B9FF0EBC4243891A1847C046002941D0FF
S11304B010B4041C4C40A44601230022002900D59A
S11304C04942002800D5404288422CD30124240705
S11304D0A14204D2814202D209011B01F8E7E400DF
S11304E0A14204D2814202D249005B00F8E788426B
S11304F001D3401A1A434C08A04202D3001B5C08E3
S113050022438C08A04202D3001B9C082243CC083F
S1130510A04202D3001BDC082243002803D01B099D
S113052001D00909E3E7101C6446002C00D54042C1
S113053010BC7047002806D003DB0020C0434008ED
S113054001E08020000607B4024802A1401802908E
S113055003BDC046190000000029EBD003B5FFF726
S1130560A7FF0EBC4243891A1847C0467047C046CD
S113057090B58BB002AFF860B9603B60BB1D1A80C8
S1130580FB68002B01D172B6FEE73B6B052B01D94A
S113059072B6FEE7BB1D1A88BB6B101C191C00F059
S11305A011FD031CBB61BB69002B00D173E0BB6967
S11305B01A6BBB1D1B88013B9B00D3187B617B69B5
S11305C0072293437B617A690723134001D072B6F3
S11305D0FEE7B869B9683A6BFB6BBC1D24880094CC
S11305E000F02EFC7969FA683B68081C111C1A1C7F
S11305F001F0ECFB021CBB691A607B6B002B02D080
S11306007B6BBA691A6001F063FC2E4B1B685A1CA1
S11306102C4B1A602C4B1B68002B09D12A4BBA694E
S11306201A60284B1B68012B0FD100F053FC0CE01F
S1130630264B1B68002B08D1234B1B68DA6A3B6BE3
S11306409A4202D8204BBA691A60214B1B685A1C83
S11306501F4B1A601E4B1A68BB691A64BB69DA6ABD
S11306601C4B1B689A4203D9BB69DA6A194B1A609E
S1130670BB69DA6A131C9B009B189B00164A9A18E4
S1130680BB690433101C191C01F0CAFC0123FB6173
S113069001F02EFC02E001235B42FB61FB69012BAC
S11306A00BD10A4B1B68002B07D0074B1B68DA6A77
S11306B03B6B9A4201D201F02BFCFB69181CBD462E
S11306C009B090BDECF0FF1F18F0FF1FF8F0FF1FFA
S11306D008F1FF1FF4F0FF1F1CF0FF1F80B584B06A
S11306E000AF78600023FB607B68002B1AD0114BAD
S11306F01B68002B01D072B6FEE700F053F80E4BD6
S11307001A687B68D318BB600C4B1B680433181C35
S113071001F0DEFCBB68181C00F01EFC00F04EF873
S1130720031CFB60FB68002B01D101F0F1FBBD460B
S113073004B080BD0CF1FF1FF0F0FF1F18F0FF1F85
S113074080B586B004AF134A134B002100910021F9
S113075001910021029100210391101C191CC8224F
S11307600023FFF705FF031C7B607B68012B09D185
S113077072B60A4B01221A60094B00221A6001F07A
S113078081FB04E07B68002B01D172B6FEE7BD4615
S113079002B080BD1D0E0000C4950000F8F0FF1FDC
S11307A0F0F0FF1F80B500AF034B1B685A1C024BCF
S11307B01A60BD4680BDC0460CF1FF1F80B582B0F3
S11307C000AF00237B60374B1B68002B01D172B64E
S11307D0FEE701F07DFB334B1B685A1E314B1A6058
S11307E0304B1B68002B56D12F4B1B68002B52D06B
S11307F02FE02E4BDB68DB683B603B681833181C2A
S113080001F066FC3B680433181C01F061FC3B6892
S1130810DA6A274B1B689A4203D93B68DA6A244B8D
S11308201A603B68DA6A131C9B009B189B00214AE0
S11308309A183B680433101C191C01F0F1FB3B6847
S1130840DA6A1D4B1B68DB6A9A4202D31B4B0122F6
S11308501A60164B1B68002BCBD1194B1B68002B5D
S113086011D00CE000F0B8F8031C002B02D0134B9D
S113087001221A60124B1B685A1E114B1A60104B4E
S11308801B68002BEED10D4B1B68012B03D10123F8
S11308907B6001F03DFB01F02BFB7B68181CBD461F
S11308A002B080BD0CF1FF1FECF0FF1FC4F0FF1F6E
S11308B0F4F0FF1F1CF0FF1F18F0FF1F00F1FF1FD3
S11308C0FCF0FF1F80B582B000AF01F001FB054BC7
S11308D01B687B6001F00CFB7B68181CBD4602B0F2
S11308E080BDC046F0F0FF1F80B500AF024B1B680F
S11308F0181CBD4680BDC046ECF0FF1F80B586B015
S113090000AFF860B9607A6000237B6106233B6125
S1130910FFF748FF2B4B1B68BA689A424BD33B69DD
S1130920013B3B617B695B01FA68D1183A69131C8E
S11309309B009B189B00244A9B18081C191C01222D
S113094000F078FB031C7A69D3187B613B69002BA8
S1130950E5D17B695B01FA68D2181C4B1B68101C3B
S1130960191C022200F066FB031C7A69D3187B6110
S11309707B695B01FA68D218154B1B68101C191CA3
S1130980022200F057FB031C7A69D3187B617B6950
S11309905B01FA68D2180F4B101C191C032200F0DB
S11309A049FB031C7A69D3187B617B68002B02D056
S11309B07B6800221A60FFF701FF7B69181CBD46A3
S11309C006B080BDECF0FF1F1CF0FF1FBCF0FF1F42
S11309D0C0F0FF1FD8F0FF1F80B586B000AF002322
S11309E07B61524B1B68002B00D08CE0504B1B6882
S11309F05A1C4F4B1A604E4B1B683B613B69002BE2
S1130A0017D14C4B1B681B68002B01D072B6FEE754
S1130A10484B1B68FB60484B1A68464B1A60464BB0
S1130A20FA681A60454B1B685A1C444B1A6000F064
S1130A30A9FB434B1B683A699A4250D300E0C04675
S1130A403C4B1B681B68002B01D1012300E00023F1
S1130A50002B04D03A4B012252421A603FE0354B3E
S1130A601B68DB68DB68BB60BB685B687B603A69FA
S1130A707B689A4203D2324B7A681A602FE0BB68D3
S1130A800433181C01F024FBBB689B6A002B04D0C0
S1130A90BB681833181C01F01BFBBB68DA6A294BCE
S1130AA01B689A4203D9BB68DA6A264B1A60BB6892
S1130AB0DA6A131C9B009B189B00234A9A18BB6894
S1130AC00433101C191C01F0ABFABB68DA6A1F4B23
S1130AD01B68DB6A9A42B2D301237B61AFE71B4BED
S1130AE01B68DA6A1849131C9B009B189B005B580F
S1130AF0012B01D901237B61154B1B68002B09D104
S1130B0007F044FF06E0124B1B685A1C104B1A6096
S1130B1007F03CFF0F4B1B68002B01D001237B61C6
S1130B207B69181CBD4606B080BDC0460CF1FF1F92
S1130B30F0F0FF1FBCF0FF1FC0F0FF1F04F1FF1F08
S1130B4000F0FF1FF4F0FF1F1CF0FF1F18F0FF1F41
S1130B50FCF0FF1F00F1FF1F80B582B000AF294BEE
S1130B601B68002B03D0284B01221A6047E0264B58
S1130B7000221A60254B1B681A68244B1B681B6BE8
S1130B809A4214D8214B1A68204B1B683433101C2A
S1130B90191C07F0F3FE0AE01D4B1B68002B01D162
S1130BA072B6FEE71A4B1B685A1E194B1A60184B93
S1130BB01A681849131C9B009B189B005B58002B58
S1130BC0EAD0134B1A68131C9B009B189B00114A14
S1130BD09B187B607B685B685A687B685A607B689B
S1130BE05A687B6808339A4204D17B685B685A6808
S1130BF07B685A607B685B68DA68044B1A60BD46A0
S1130C0002B080BD0CF1FF1F00F1FF1F18F0FF1FA1
S1130C10F4F0FF1F1CF0FF1F80B584B000AF7860B4
S1130C2039607B68002B01D172B6FEE7124B1B685A
S1130C3018337A68101C191C01F014FA0E4B1B6847
S1130C400433181C01F044FA3B68013308D10A4B01
S1130C501B680433094A101C191C01F0E1F908E06F
S1130C60074B1A683B68D318FB60FB68181C00F03C
S1130C7073F9BD4604B080BD18F0FF1FD8F0FF1F04
S1130C80F0F0FF1F80B584B000AF78607B68DB684C
S1130C90DB68BB60BB68002B01D172B6FEE7BB68A2
S1130CA01833181C01F014FA1E4B1B68002B1DD1BD
S1130CB0BB680433181C01F00BFABB68DA6A1A4BE0
S1130CC01B689A4203D9BB68DA6A174B1A60BB687F
S1130CD0DA6A131C9B009B189B00144A9A18BB6881
S1130CE00433101C191C01F09BF906E0BB6818338F
S1130CF00F4A101C191C01F093F9BB68DA6A0D4BFA
S1130D001B68DB6A9A4205D90123FB600A4B012266
S1130D101A6001E00023FB60FB68181CBD4604B0A8
S1130D2080BDC0460CF1FF1FF4F0FF1F1CF0FF1F35
S1130D30C4F0FF1F18F0FF1F00F1FF1F80B582B041
S1130D4000AF78607B68002B01D172B6FEE7054BDB
S1130D501A687B681A60044B1A687B685A60BD463F
S1130D6002B080BD04F1FF1FF0F0FF1F80B584B016
S1130D7000AF786039607B68002B01D172B6FEE762
S1130D803B68002B01D172B6FEE701F0A1F81C4BC1
S1130D901B68BB603B681B68013302D10023FB6006
S1130DA027E07B681A68174B1B689A4207D07B6858
S1130DB05A68BB689A4202D80123FB6019E07B6839
S1130DC05B68BA68D21A3B681B689A420FD23B68C8
S1130DD01A687B685968BB68CB1AD2183B681A60DA
S1130DE07B68181CFFF7AAFF0023FB6001E00123C6
S1130DF0FB6001F07DF8FB68181CBD4604B080BDA3
S1130E00F0F0FF1F04F1FF1F80B500AF024B012279
S1130E101A60BD4680BDC04600F1FF1F80B582B098
S1130E2000AF786000F094F8044B1B68012B01D9E3
S1130E3001F06EF807F0B0FDF4E7C0461CF0FF1FA8
S1130E4080B586B000AFF860B9607A603B6000237B
S1130E507B6112E0BA687B69D3181A78F86830238A
S1130E6079694118CB181A71BA687B69D3181B7851
S1130E70002B06D07B6901337B617B690B2BE9D99D
S1130E8000E0C046FA683F230021D1547B68052B5B
S1130E9001D905237B60FB687A68DA62FB687A68AB
S1130EA09A64FB680433181C01F0B0F8FB6818332B
S1130EB0181C01F0ABF8FB68FA681A617B6806221B
S1130EC0D21AFB689A61FB68FA685A62BD4606B09A
S1130ED080BDC04680B582B000AF00237B600CE0CB
S1130EE07A68131C9B009B189B00124A9B18181CC1
S1130EF001F06EF87B6801337B607B68052BEFD9CA
S1130F000D4B181C01F064F80C4B181C01F060F830
S1130F100B4B181C01F05CF80A4B181C01F058F834
S1130F20094B054A1A60094B044A1A60BD4602B0CF
S1130F3080BDC0461CF0FF1F94F0FF1FA8F0FF1FE8
S1130F40C4F0FF1FD8F0FF1FBCF0FF1FC0F0FF1F4D
S1130F5080B500AFBD4680BD80B582B000AF78607B
S1130F60134B1B687A685A60124B1B687A689A4262
S1130F7009D2114B1A680E4B1B680433101C191C40
S1130F8001F070F810E00D4B1A68094B1B6804332C
S1130F90101C191C01F066F8094B1B687A689A4208
S1130FA002D2074B7A681A60BD4602B080BDC046C3
S1130FB018F0FF1FF0F0FF1FC0F0FF1FBCF0FF1F71
S1130FC000F0FF1F80B584B000AF021C3960BB1D68
S1130FD01A804C2001F0A4F8031CFB60FB68002B72
S1130FE022D03B68002B07D1BB1D1B889B00181C1B
S1130FF001F096F8021C00E03A68FB681A63FB688B
S11310001B6B002B06D1FB68181C01F01FF9002391
S1131010FB6009E0FB681A6BBB1D1B889B00101C5E
S1131020A5211A1C08F0B9F9FB68181CBD4604B0C8
S113103080BDC04690B58BB000AFF860B960FB1DB1
S11310401A7000237B62BB681B68002B00D17AE016
S1131050BB683B623B6A5B685A683B6A5A603B6A9E
S11310605A683B6A08339A4204D13B6A5B685A68FF
S11310703B6A5A603B6A5B68DB68FB61BB68BB61C7
S1131080BB695B685A68BB695A60BB695A68BB69CB
S113109008339A4204D1BB695B685A68BB695A60D9
S11310A0BB695B68DB687B617B6A5B01FA68D318A8
S11310B07A691A607B6A5B01FA68D3187A693432F8
S11310C05A607B6A5B01FA68D3187A69126C9A6079
S11310D07B6A5B01FA68D318FA1D12781A737B6A6B
S11310E05B01FA68D3187A69D26A1A61FB1D1B780E
S11310F0032B09D17B699B6A002B05D07B6A5B01BA
S1131100FA68D31802221A737B6A5B01FA68D3184F
S11311107A69926C5A617B6A5B01FA68D31800227F
S11311209A617B6A5B01FA68D4187B691B6B181C93
S113113000F00EF8031CA3837B6A01337B627A6997
S1131140FB699A429AD17B6A181CBD460BB090BDCC
S113115080B584B000AF78600023FB6005E07B6855
S113116001337B60FB680133FB607B681B78A52B34
S1131170F5D0FB689B08FB60FB689BB2181CBD465E
S113118004B080BD80B582B000AF0D4B1B681B68F6
S1131190002B01D1012300E00023002B04D0094BD4
S11311A0012252421A6008E0054B1B68DB68DB68C9
S11311B07B607B685A68034B1A60BD4602B080BDF1
S11311C0BCF0FF1F00F0FF1F80B582B000AF044BDE
S11311D01B687B607B68181CBD4602B080BDC0469E
S11311E018F0FF1F80B582B000AF0A4B1B68002BBC
S11311F002D101237B6008E0074B1B68002B02D15E
S113120002237B6001E000237B607B68181CBD46E1
S113121002B080BDF8F0FF1F0CF1FF1F80B584B051
S113122000AF78607B68FB607B68002B4AD0FB686A
S1131230DA6A264B1B68DB6A9A4243D2FB689B69D5
S1131240002B06DB214B1B68DB6A0622D21AFB68E3
S11312509A61FB685969FB68DA6A131C9B009B1846
S11312609B001B4A9B18994201D1012300E00023F3
S1131270002B22D0FB680433181C00F029FF134B09
S11312801B68DA6AFB68DA62FB68DA6A114B1B686E
S11312909A4203D9FB68DA6A0E4B1A60FB68DA6A71
S11312A0131C9B009B189B00094A9A18FB68043383
S11312B0101C191C00F0B4FE04E0044B1B68DA6A2D
S11312C0FB68DA62BD4604B080BDC04618F0FF1F5B
S11312D01CF0FF1FF4F0FF1F80B584B000AF7860EE
S11312E07B68FB607B68002B30D0FB68DA6AFB68A4
S11312F09B6C9A422AD0FB680433181C00F0E8FE69
S1131300FB689A6CFB68DA62FB689B69002B05DB5F
S1131310FB68DB6A0622D21AFB689A61FB68DA6A08
S11313200C4B1B689A4203D9FB68DA6A094B1A60B2
S1131330FB68DA6A131C9B009B189B00064A9A18E8
S1131340FB680433101C191C00F06AFEBD4604B08F
S113135080BDC046F4F0FF1F1CF0FF1F80B586B0AF
S113136000AF786039607B6800221A70584B1B68A4
S1131370FB60574B1B685B01181C00F0D1FE031C7B
S11313803B613B69002B00D19FE0FB683A69101C6C
S1131390191C0022FFF7B2FA031CFB600023BB6098
S11313A08AE0BB685B013A69D3181B7B022B0DD022
S11313B002DC012B05D018E0032B0CD0042B0FD03A
S11313C013E03B1C173352221A7013E03B1C1733F3
S11313D042221A700EE03B1C173353221A7009E0A4
S11313E03B1C173344221A7004E03B1C17330022C1
S11313F01A70C046BB685B013A69D3185B687968A8
S11314003A68081C111C1A1C00F0E2FF79683A685B
S1131410304B081C111C1A1C00F0DAFF79683A687A
S11314203B1C17331B78081C111C1A1C01F002F812
S11314307A683B68101C191C092200F0FBFFBB688A
S11314405B013A69D3181B6979683A68081C111C56
S11314501A1C01F09FFA7A683B68101C191C0922B7
S113146000F0E8FFBB685B013A69D3189B8B79688D
S11314703A68081C111C1A1C01F08CFA7A683B6843
S1131480101C191C092200F0D5FFBB685B013A69E6
S1131490D3189B6879683A68081C111C1A1C01F05F
S11314A079FA79683A680C4B081C111C1A1C00F074
S11314B08FFFBB680133BB60BA68FB689A4200D2F5
S11314C06FE73B69181C00F0C1FEBD4606B080BD45
S11314D0ECF0FF1FCC950000D095000080B584B0DF
S11314E000AF786039607B68FB60FB68002B01D13A
S11314F072B6FEE700F0ECFCFB681A68FB68D96B77
S1131500FB681B6C4B43D218FB685A60FB680022D3
S11315109A63FB681A68FB689A60FB681A68FB6840
S1131520DB6B591EFB681B6C4B43D218FB68DA60FB
S1131530FB68012252425A64FB68012252429A64B7
S11315403B68002B0ED1FB681B69002B14D0FB6891
S11315501033181CFFF796FB031C012B0CD100F071
S1131560D7FC09E0FB681033181C00F031FDFB6860
S11315702433181C00F02CFD00F0BAFC0123181CC5
S1131580BD4604B080BDC04680B588B000AFF860E9
S1131590B960FB1D1A700023FB61FB68002B2ED081
S11315A0542000F0BDFD031CBB61BB69002B26D099
S11315B0FB68BA68534301337B617B69181C00F0F4
S11315C0AFFD021CBB691A60BB691B68002B12D0FB
S11315D0BB69FA68DA63BB69BA681A64BB69181C28
S11315E00121FFF77BFFBA69F91D50230978D15413
S11315F0BB69FB6103E0BB69181C00F027FEFB69B3
S1131600002B01D172B6FEE7FB69181CBD4608B079
S113161080BDC04680B584B000AF021CFB1D1A70AB
S1131620542000F07DFD031CFB60FB68002B32D0CE
S1131630FB6800225A60FB6800221A60FB680022E3
S11316409A60FB680022DA60FB6800229A63FB68F8
S11316500122DA63FB6800221A64FB680122524209
S11316605A64FB68012252429A64FA68F91D5023B5
S11316700978D154FB681033181C00F0A9FCFB68EE
S11316802433181C00F0A4FCFB68181C0021002261
S1131690002300F069F8FB68002B01D172B6FEE765
S11316A0FB68181CBD4604B080BDC04690B585B02B
S11316B000AF78607B68BB60BB68002B01D172B659
S11316C0FEE7BB685C68FFF77FFD031C9C4212D1F8
S11316D0BB68DB685A1EBB68DA60BB68DB68002B3A
S11316E006D1BB68181C00210022002300F03CF83E
S11316F00123FB6001E00023FB60FB68181CBD466E
S113170005B090BD90B585B000AF786039607B6856
S1131710BB60BB68002B01D172B6FEE7BB685C6896
S1131720FFF752FD031C9C4207D1BB68DB685A1CBF
S1131730BB68DA600123FB6011E0BA683B68101CE7
S113174000211A1C002300F035F9031CFB60FB6820
S1131750012B04D1BB68DB685A1CBB68DA60FB68E8
S1131760181CBD4605B090BD80B588B000AFF860C8
S1131770B9607A603B600023FB61FB68BB61BB69B5
S1131780002B01D172B6FEE7BB68002B03D1BB6905
S11317901B6C002B01D1012300E00023002B01D19D
S11317A072B6FEE73B68022B03D1BB69DB6B012BEE
S11317B001D1012300E00023002B01D172B6FEE722
S11317C0FFF710FD031C002B02D17B68002B01D115
S11317D0012300E00023002B02D172B6FEE7C046CD
S11317E000F076FBBB699A6BBB69DB6B9A4202D350
S11317F03B68022B19D1B969BA683B68081C111CF3
S11318001A1C00F0CBF9BB695B6A002B09D0BB69D9
S11318102433181CFFF736FA031C012B01D100F006
S113182077FB00F065FB012359E07B68002B03D1B3
S113183000F05EFB002352E0FB69002B06D13B1C49
S11318401033181CFFF77AFA0123FB6100F050FBF8
S1131850FEF7A8FF00F03CFBBB695B6C013302D1CF
S1131860BB6900225A64BB699B6C013302D1BB691A
S113187000229A6400F03CFB3A1C10323B1D101C01
S1131880191CFFF773FA031C002B21D1BB69181C28
S113189000F078FA031C002B13D0BB691A1C103219
S11318A07B68101C191CFFF7B7F9BB69181C00F002
S11318B007FAFEF783FF031C002B90D100F028FBEE
S11318C08DE7BB69181C00F0FBF9FEF777FF86E78C
S11318D0BB69181C00F0F4F9FEF770FF0023181C14
S11318E0BD4608B080BDC04680B588B000AFF86082
S11318F0B9607A603B60FB68BB61BB69002B01D1B6
S113190072B6FEE7BB68002B03D1BB691B6C002BCE
S113191001D1012300E00023002B01D172B6FEE7C0
S11319203B68022B03D1BB69DB6B012B01D1012383
S113193000E00023002B01D172B6FEE700237B6197
S113194072B6BB699A6BBB69DB6B9A4202D33B6884
S1131950022B26D1B969BA683B68081C111C1A1CF1
S113196000F01CF9BB699B6C013312D1BB695B6A43
S1131970002B13D0BB692433181CFFF783F9031C15
S1131980002B0BD07B68002B08D07B6801221A60E7
S113199004E0BB699B6C5A1CBB699A640123FB611C
S11319A001E00023FB6162B6FB69181CBD4608B068
S11319B080BDC04680B58AB000AFF860B9607A6077
S11319C03B6000237B62FB683B623B6A002B01D1D6
S11319D072B6FEE7BB68002B03D13B6A1B6C002B7D
S11319E001D1012300E00023002B01D172B6FEE7F0
S11319F0FFF7F8FB031C002B02D17B68002B01D1FD
S1131A00012300E00023002B02D172B6FEE7C0469A
S1131A1000F05EFA3B6A9B6B002B3DD03B6ADB68AF
S1131A20FB613A6ABB68101C191C00F021F93B6881
S1131A30002B1CD13B6A9B6B5A1E3B6A9A633B6A20
S1131A401B68002B04D1FFF7BFFB021C3B6A5A60E2
S1131A503B6A1B69002B1BD03B6A1033181CFFF731
S1131A6011F9031C012B13D100F052FA10E03B6A68
S1131A70FA69DA603B6A5B6A002B09D03B6A24335B
S1131A80181CFFF7FFF8031C002B01D000F040FAEC
S1131A9000F02EFA012367E07B68002B03D100F0ED
S1131AA027FA002360E07B6A002B06D13B1C143329
S1131AB0181CFFF743F901237B6200F019FAFEF7C3
S1131AC071FE00F005FA3B6A5B6C013302D13B6A9C
S1131AD000225A643B6A9B6C013302D13B6A0022A8
S1131AE09A6400F005FA3A1C14323B1D101C191CB0
S1131AF0FFF73CF9031C002B2FD13B6A181C00F0A4
S1131B002BF9031C002B21D03B6A1B68002B08D146
S1131B1000F0DEF93B6A5B68181CFFF77FFB00F0FE
S1131B20E7F93B6A1A1C24327B68101C191CFFF766
S1131B3073F83B6A181C00F0C3F8FEF73FFE031C61
S1131B40002B00D063E700F0E3F960E73B6A181C60
S1131B5000F0B6F8FEF732FE59E73B6A181C00F0B5
S1131B60AFF8FEF72BFE0023181CBD460AB080BD5B
S1131B7080B584B000AF78607B68002B01D172B669
S1131B80FEE700F0A5F97B689B6BFB6000F0B0F901
S1131B90FB68181CBD4604B080BDC04680B584B047
S1131BA000AFF860B9607A60FB681B6C002B0CD145
S1131BB0FB681B68002B53D1FB685B68181CFFF79C
S1131BC08BFBFB6800225A604AE07B68002B1BD128
S1131BD0FB689968FB681B6CBA68081C111C1A1C0A
S1131BE007F0D2FBFB689A68FB681B6CD218FB6891
S1131BF09A60FB689A68FB685B689A4230D3FB681A
S1131C001A68FB689A602BE0FB68D968FB681B6C58
S1131C10BA68081C111C1A1C07F0B6FBFB68DA68CA
S1131C20FB681B6C5B42D218FB68DA60FB68DA68FD
S1131C30FB681B689A4207D2FB685A68FB681B6CF6
S1131C405B42D218FB68DA607B68022B08D1FB6820
S1131C509B6B002B04D0FB689B6B5A1EFB689A633A
S1131C60FB689B6B5A1CFB689A63BD4604B080BD3D
S1131C7080B582B000AF786039607B681B68002B48
S1131C801AD07B68DA687B681B6CD2187B68DA60D0
S1131C907B68DA687B685B689A4203D37B681A685E
S1131CA07B68DA607B68DA687B681B6C3968081CBF
S1131CB0111C1A1C07F068FBBD4602B080BDC0466B
S1131CC080B582B000AF786000F002F912E07B6862
S1131CD05B6A002B13D07B682433181CFEF7D2FFF9
S1131CE0031C002B01D0FFF78FF87B689B6C5A1EF6
S1131CF07B689A647B689B6C002BE8DC00E0C04640
S1131D007B68012252429A6400F0F2F800F0E0F895
S1131D1012E07B681B69002B13D07B681033181CFE
S1131D20FEF7B0FF031C002B01D0FFF76DF87B68B2
S1131D305B6C5A1E7B685A647B685B6C002BE8DC26
S1131D4000E0C0467B68012252425A6400F0D0F899
S1131D50BD4602B080BDC04680B584B000AF786097
S1131D6000F0B6F87B689B6B002B02D10123FB606B
S1131D7001E00023FB6000F0BBF8FB68181CBD46C3
S1131D8004B080BD80B584B000AF786000F0A0F8E6
S1131D907B689A6B7B68DB6B9A4202D10123FB6000
S1131DA001E00023FB6000F0A3F8FB68181CBD46AB
S1131DB004B080BD80B500AF034B1B68013301D074
S1131DC072B6FEE772B6FEE704F0FF1F80B584B07A
S1131DD000AFF860B9607A60FB68043BFB60FB68A5
S1131DE0802252041A60FB68043BFB60BA68FB68FB
S1131DF01A60FB68043BFB60084AFB681A60FB68D6
S1131E00143BFB607A68FB681A60FB68203BFB604C
S1131E10FB68181CBD4604B080BDC046B51D00005B
S1131E2080B500AF084B084A1268C02109060A436E
S1131E301A60064B064A1A60064B00221A60064BCB
S1131E4007221A60BD4680BD20ED00E014E000E0EA
S1131E507FBB000018E000E010E000E080B500AFB8
S1131E60024B07221A60BD4680BDC04610E000E068
S1131E7080B500AF024B06221A60BD4680BDC04645
S1131E8010E000E080B500AF0E4B0E4A1268C0218E
S1131E9009040A431A600C4B00221A60FFF7C0FFC2
S1131EA0FFF7DCFF094B181C07F07EFB031C002B1B
S1131EB001D0002302E000F047F80023181CBD46BF
S1131EC080BDC04620ED00E004F0FF1F10F1FF1FAD
S1131ED080B500AF72B6054B1B685A1C034B1A60E1
S1131EE0BFF34F8FBFF36F8FBD4680BD04F0FF1F5C
S1131EF080B500AF054B1B685A1E044B1A60034B98
S1131F001B68002B00D162B6BD4680BD04F0FF1FE4
S1131F1080B500AF044B802252051A60BFF34F8F87
S1131F20BFF36F8FBD4680BD04ED00E080B500AF08
S1131F3072B6FEF751FD031C002B01D0FFF7E8FF3A
S1131F4062B6BD4680BDC04680B500AF0448006897
S1131F50006880F3088862B600DFC046BD4680BDD5
S1131F6008ED00E0084B196808681030F0C8A04676
S1131F70A946B246BB4680F309882038F0C87146AA
S1131F800D2001430847C04618F0FF1FEFF30980F6
S1131F900E4B1A6820381060F0C044464D46564631
S1131FA05F46F0C008B572B6FEF7D6FD62B60CBC4B
S1131FB0116808681030F0C8A046A946B246BB466E
S1131FC080F309882038F0C81847C04618F0FF1F6E
S1131FD080B582B000AF78607B681A1C08327B68D9
S1131FE05A607B68012252429A607B681A1C08324C
S1131FF07B68DA607B681A1C08327B681A617B682C
S113200000221A60BD4602B080BDC04680B582B0D1
S113201000AF78607B6800221A61BD4602B080BDC3
S113202080B584B000AF786039607B685B68FB6022
S11320303B68FA685A60FB689A683B689A60FB6878
S11320409B683A685A60FB683A689A603B687A68A9
S11320501A617B681B685A1C7B681A60BD4604B011
S113206080BDC04680B584B000AF786039603B68FD
S11320701B68BB60BB68013303D17B681B69FB60D1
S11320800CE07B680833FB6002E0FB685B68FB6084
S1132090FB685B681A68BB689A42F6D9FB685A68A1
S11320A03B685A603B685B683A689A603B68FA68C8
S11320B09A60FB683A685A603B687A681A617B6880
S11320C01B685A1C7B681A60BD4604B080BDC046BC
S11320D080B584B000AF78607B681B69FB607B6867
S11320E05B687A6892689A607B689B687A685268D1
S11320F05A60FB685A687B689A4203D17B689A6885
S1132100FB685A607B6800221A61FB681B685A1ED0
S1132110FB681A60FB681B68181CBD4604B080BDD0
S113212080B588B000AF786000237B61FEF73AFB8E
S1132130404B1B68002B04D100F0CEF83D4B01222C
S11321401A607B68002B0DD03B4B1B887A68D31830
S11321507B607A680723134004D07B68072293438B
S113216008337B607B68002B58D07A68334B9A42E3
S113217054D8334BBB61324B1B68FB6104E0FB69F1
S1132180BB61FB691B68FB61FB695A687B689A4207
S113219003D2FB691B68002BF1D1FA69294B9A42DF
S11321A03CD0BB691A68244B1B88D3187B61FB693C
S11321B01A68BB691A60FB695A687B68D21A1E4B9D
S11321C01B885B009A4222D9FA697B68D318FB60AA
S11321D0FB695A687B68D21AFB685A60FB697A68A3
S11321E05A60FB685B68BB60154B3B6102E03B696E
S11321F01B683B613B691B685A68BB689A42F6D30B
S11322003B691A68FB681A603B69FA681A600E4BEE
S11322101A68FB695B68D21A0B4B1A60FEF7CEFA98
S11322207B69002B01D106F0BBFB7B69181CBD4602
S113223008B080BD7018002068A1000007270000C6
S1132240601800206818002008F0FF1F80B586B0D1
S113225000AF78607B683B617B68002B28D0164B0D
S11322601B885B423A69D3183B613B69FB60FEF70C
S113227099FAFB685B68BB60104B7B6102E07B6989
S11322801B687B617B691B685A68BB689A42F6D3FA
S11322907B691A68FB681A607B69FA681A60FB68D4
S11322A05A68074B1B68D218054B1A60FEF786FA6A
S11322B0BD4606B080BDC04668A10000601800207D
S11322C008F0FF1F80B500AF024B1B68181CBD4609
S11322D080BDC04608F0FF1F80B582B000AF0D4B33
S11322E0072293437B600C4B7A681A600A4B0022E6
S11322F05A600A4B0A4A5A60084B00221A607B68EB
S11323003B603B68064A5A603B68044A1A60BD4613
S113231002B080BD58F1FF1F60180020681800202B
S113232008270000C046C046C04670470020C0468B
S1132330C046C046C046C04601300928F7D9C04649
S11323407047C04680B582B000AF021CBB1D1A8026
S113235006E0FFF7EBFFBB1DBA1D1288643A1A8032
S1132360BB1D1B88642BF4D806E0FFF7DBFFBB1D05
S1132370BA1D12880A3A1A80BB1D1B880A2BF4D88E
S1132380BD4602B080BDC04680B584B000AFF860E1
S1132390B9607A60BB68013BBB600CE07B681A786B
S11323A0FB681A70FB680133FB607B6801337B6058
S11323B0BB68013BBB60BB68002B03D07B681B7808
S11323C0002BEBD1FB6800221A70BD4604B080BD1F
S11323D080B584B000AFF860B9607A60BB68013B37
S11323E0BB6005E0FB680133FB60BB68013BBB607D
S11323F0BB68002B11D0FB681B78002BF2D10CE0DA
S11324007B681A78FB681A70FB680133FB607B6891
S113241001337B60BB68013BBB60BB68002B03D00E
S11324207B681B78002BEBD1FB6800221A70BD4639
S113243004B080BD80B584B000AFF860B960FB1D06
S11324401A70BB68013BBB6005E0FB680133FB60AD
S1132450BB68013BBB60BB68002B03D0FB681B78E7
S1132460002BF2D1BB68002B06D0FB68FA1D127852
S11324701A70FB680133FB60FB6800221A70BD46CA
S113248004B080BD80B584B000AFF860B960FB1DB6
S11324901A70FB1D1B789BB2F968BA68081C111CE2
S11324A01A1C00F019F8BD4604B080BD80B584B094
S11324B000AFF860B960FB1D1A70FB1D1B785BB29E
S11324C09BB2F968BA681BB2081C111C1A1C00F0F4
S11324D09FF8BD4604B080BD90B589B000AFF860E8
S11324E0B960BB1D1A80FB68BB613B1C1F33002213
S11324F01A70BB68013BBB60BB1D1B88002B38D125
S1132500BB68002B35D03B1C1F331B78BA69D3182A
S113251030221A703B1C1F333A1C1F3212780132CE
S11325201A70BB68013BBB6023E03B1C1F331B7864
S1132530BA69D418BB1D1B88181C0A21FDF7ACFF0F
S11325400B1C9BB2DBB23033DBB223703B1C1F335A
S11325503A1C1F32127801321A70BB68013BBB600F
S1132560BC1DBB1D1B88181C0A21FDF751FF031C51
S11325702380BB1D1B88002B02D0BB68002BD4D149
S11325803B1C1E3300221A702EE03B1C1E331B78AA
S1132590BA69D2183B1C173312781A703B1C1E33CD
S11325A01B78BA69D3183A1C1F3211783A1C1E32B0
S11325B012788A1A013AB9698A1812781A703B1C7F
S11325C01F331A783B1C1E331B78D31A013BBA699C
S11325D0D3183A1C173212781A703B1C1E333A1C5B
S11325E01E32127801321A703B1C1F331B785B08B1
S11325F0DBB23A1C1E3212789A42C6D33B1C1F33FC
S11326001B78BA69D31800221A70BD4609B090BD70
S113261090B589B000AFF860B960BB1D1A80FB6843
S1132620BB613B1C1F3300221A70BB1D1B88DB0BD4
S1132630DAB23B1C17331A70BB1D00215A5E614B82
S11326409A4208D1F968BA685F4B081C111C1A1C1D
S1132650FFF79AFEB3E0BB68013BBB603B1C17333A
S11326601B78002B05D0BB1D1B885B429AB2BB1D97
S11326701A80BB1D00229B5E002B3AD1BB68002B45
S113268037D03B1C1F331B78BA69D31830221A7019
S11326903B1C1F333A1C1F32127801321A70BB687C
S11326A0013BBB6025E03B1C1F331B78BA69D4187F
S11326B0BB1D00215B5E181C0A21FDF74DFF0B1C9E
S11326C09BB2DBB23033DBB223703B1C1F333A1CAA
S11326D01F32127801321A70BB68013BBB60BC1D0B
S11326E0BB1D00229B5E181C0A21FDF7DFFE031CA4
S11326F02380BB1D00215B5E002B02DDBB68002B29
S1132700D1D13B1C17331B78002B13D0BB68002B93
S113271010D03B1C1F331B78BA69D3182D221A70B2
S11327203B1C1F333A1C1F32127801321A70BB68EB
S1132730013BBB603B1C1E3300221A702EE03B1C85
S11327401E331B78BA69D2183B1C163312781A70E0
S11327503B1C1E331B78BA69D3183A1C1F321178FC
S11327603A1C1E3212788A1A013AB9698A18127808
S11327701A703B1C1F331A783B1C1E331B78D31A68
S1132780013BBA69D3183A1C163212781A703B1CF2
S11327901E333A1C1E32127801321A703B1C1F334E
S11327A01B785B08DBB23A1C1E3212789A42C6D3FD
S11327B03B1C1F331B78BA69D31800221A70BD461C
S11327C009B090BD0080FFFFD495000080B586B0AD
S11327D000AFF860B960FB1D1A703A1C1432FB1D7F
S11327E01B78101C04211A1CFFF74CFEF968BA6808
S11327F03B1C1433081C111C1A1CFFF7E9FDBD46D1
S113280006B080BD80B586B000AFF860B960FB1D2E
S11328101A703A1C1032FB1D1B785BB2101C052188
S11328201A1CFFF743FEF968BA683B1C1033081CF6
S1132830111C1A1CFFF7CCFDBD4606B080BDC04676
S113284080B586B000AFF860B960BB1D1A803A1C31
S11328501032BB1D00215B5E101C07211A1CFFF700
S1132860D7FEF968BA683B1C1033081C111C1A1CEB
S1132870FFF7AEFDBD4606B080BDC04680B586B04C
S113288000AFF860B960FB1D1A703B1C14330022C2
S11328909A703B1C1733FA1D11780F220A401A70E4
S11328A03B1C17331B78092B01D8302300E0372356
S11328B03A1C173212789B18DAB23B1C14335A7044
S11328C03B1C1733FA1D127812091A703B1C17337C
S11328D01B78092B01D8302300E037233A1C173228
S11328E012789B18DAB23B1C14331A70F968BA6870
S11328F03B1C1433081C111C1A1CFFF769FDBD4650
S113290006B080BD80B586B000AFF860B960BB1D6D
S11329101A803B1C103300221A713B1C173303220C
S11329201A70BB1D1B88D9B23B1C16330F220A40F8
S11329301A703B1C173300229A563B1C16331B7823
S1132940092B01D8302300E03723391C16310978CC
S11329505B18D9B23B1C10339954BB1DBA1D1288A5
S113296012091A803B1C17333A1C17321278013AA9
S11329701A703B1C17331B787F2BD2D9F968BA68BD
S11329803B1C1033081C111C1A1CFFF721FDBD460B
S113299006B080BD80B588B000AFF860B9607A60D9
S11329A03A1C14327B68101C0B211A1C00F00CF822
S11329B0F968BA683B1C1433081C111C1A1CFFF775
S11329C007FDBD4608B080BD90B589B000AFF86082
S11329D0B9607A60FB68BB613B1C1F3300221A702C
S11329E0BB68013BBB607B68002B34D1BB68002B08
S11329F031D03B1C1F331B78BA69D31830221A70AC
S1132A003B1C1F333A1C1F32127801321A70BB6808
S1132A10013BBB601FE03B1C1F331B78BA69D41811
S1132A207B68181C0A21FDF737FD0B1CDBB2303321
S1132A30DBB223703B1C1F333A1C1F321278013265
S1132A401A70BB68013BBB607B68181C0A21FDF748
S1132A50DFFC031C7B607B68002B02D0BB68002B6F
S1132A60D9D13B1C1E3300221A702EE03B1C1E33AE
S1132A701B78BA69D2183B1C173312781A703B1CA6
S1132A801E331B78BA69D3183A1C1F3211783A1CCA
S1132A901E3212788A1A013AB9698A1812781A70A1
S1132AA03B1C1F331A783B1C1E331B78D31A013B83
S1132AB0BA69D3183A1C173212781A703B1C1E33A9
S1132AC03A1C1E32127801321A703B1C1F331B78D9
S1132AD05B08DBB23A1C1E3212789A42C6D33B1C06
S1132AE01F331B78BA69D31800221A70BD4609B087
S1132AF090BDC04680B584B000AF786039603B1C9F
S1132B000F3304221A707B681B68BB6002E0BB6849
S1132B100133BB60BB681B78202BF8D03B680022D4
S1132B201A7018E03B681B781A1C9200D3185B00DB
S1132B30DAB2BB681B78D318DBB2303BDAB23B683D
S1132B401A703B1C0F333A1C0F321278013A1A7078
S1132B50BB680133BB60BB681B782F2B08D9BB68EB
S1132B601B78392B04D83B1C0F331B78002BD9D18D
S1132B703B1C0F331B78002B01D104230AE03B1CC0
S1132B800F331B78042B01D11B2303E07B68BA6845
S1132B901A600023181CBD4604B080BD90B587B0F0
S1132BA000AF786039607B681B683B6102E03B6979
S1132BB001333B613B691B78202BF8D03B68002232
S1132BC01A703B691B782D2B07D13B1C173301224C
S1132BD01A703B6901333B6103E03B1C173300224D
S1132BE01A703C1C16343A1C10323B1C0F33101C58
S1132BF0191CFFF77FFF031C23703B1C16331B7843
S1132C00002B03D03B1C16331B7817E03B1C1733F7
S1132C101B78002B08D03B1C0F331B785B42DBB2C4
S1132C20DAB23B681A7005E03B1C0F331B78DAB24A
S1132C303B681A703A697B681A600023181CBD4609
S1132C4007B090BD80B584B000AF78607B681B6826
S1132C50FB6002E0FB680133FB60FB681B78202B00
S1132C60F8D0FB681B78302B01D01B230FE0FB68E6
S1132C700133FB60FB681B78782B01D01B2306E033
S1132C80FB680133FB607B68FA681A600023181C38
S1132C90BD4604B080BDC04680B584B000AF786046
S1132CA039607B681A683B1C0F3312781A703B1C1E
S1132CB00F331B782F2B12D93B1C0F331B78392B66
S1132CC00DD83B1C0F331B78303BDAB23B681A70CB
S1132CD07B681B685A1C7B681A60002330E03B1C2D
S1132CE00F331B78602B12D93B1C0F331B78662BD8
S1132CF00DD83B1C0F331B78573BDAB23B681A7074
S1132D007B681B685A1C7B681A60002318E03B1C14
S1132D100F331B78402B12D93B1C0F331B78462BE7
S1132D200DD83B1C0F331B78373BDAB23B681A7063
S1132D307B681B685A1C7B681A60002300E01B2315
S1132D40181CBD4604B080BD80B586B000AF786065
S1132D5039603B1C173303221A707B681B683B6184
S1132D603B1C1033181CFFF76DFF031C002B01D014
S1132D701B2330E03B6800221A7011E03B681B788B
S1132D801B01DAB23B1C0F331B78D318DAB23B6851
S1132D901A703B1C17333A1C17321278013A1A7016
S1132DA03A1C10323B1C0F33101C191CFFF774FF24
S1132DB0031C002B04D13B1C17331B78002BDDD1E3
S1132DC03B1C17331B78002B01D1042303E03A6921
S1132DD07B681A600023181CBD4606B080BDC0463F
S1132DE080B584B000AF3A60FB1D021C1A703B1D15
S1132DF00A1C1A803B1C0F33EFF3108072B6187054
S1132E00FB1D1A780A4BD200391D0988D152FB1DCB
S1132E101B78074ADB00D31804333A681A603B1C5A
S1132E200F33187880F31088BD4604B080BDC046C7
S1132E307418002080B584B000AF3B1C0E33002210
S1132E401A703B1C0F3300221A703EE0FB1DEFF397
S1132E50108072B618703B1C0F331B78214ADB00BC
S1132E60D31804331B68002B24D03B1C0F331A786F
S1132E701C4BD200D35A002B1CD13B1C0F331B78A4
S1132E80184ADB00D31804331B68BB603B1C0F33A8
S1132E901B78144ADB00D318043300221A60FB1D8C
S1132EA0187880F31088BB6898473B1C0E330122C6
S1132EB01A7003E0FB1D187880F310883B1C0F3355
S1132EC03A1C0F32127801321A703B1C0F331B78F4
S1132ED0012BBBD93B1C0E331B78181CBD4604B018
S1132EE080BDC0467418002080B582B000AFFB1DC1
S1132EF000221A701EE0BB1DEFF3108072B618702A
S1132F00FB1D1A78124BD200D35A002B09D0FB1D9B
S1132F101B780F4AD9008A5A013A91B20C4ADB0055
S1132F209952BB1D187880F31088FB1DFA1D127886
S1132F3001321A70FB1D1B78012BDCD9C046FFF748
S1132F4079FF031C002BFAD1BD4602B080BDC046F8
S1132F507418002080B582B000AFFB1D00221A70E7
S1132F6012E0FB1D1A780C4BD2000021D152FB1D3C
S1132F701B78094ADB00D318043300221A60FB1DB6
S1132F80FA1D127801321A70FB1D1B78012BE8D947
S1132F90BD4602B080BDC0467418002080B584B020
S1132FA000AF7860364BFB60FB687A689A61354BFA
S1132FB0FA681A60FB6800221A60FB6800229A8093
S1132FC0FB6800229A81FB6800229A60FB68002259
S1132FD0DA81FB6800229A82FB6800221A612A4A7D
S1132FE029492A4BCB588021C9031943274BD15077
S1132FF0274A2749C2239B00C958264B0B408021EE
S113300009041943C2239B00D150214B204A126862
S11330108021C9000A431A601F4B1F4AD1681F4A06
S11330200A40802189000A43DA601B4B1A4A9168DE
S11330301A4A0A40802189000A439A60164B164AAC
S11330405168164A0A40802189000A435A60144B89
S113305012221A70124B10225A70114B21229A70AC
S11330600F4B0F4A1278D2B240210A43D2B21A70DF
S11330700C4BFA689A62FB68181CBD4604B080BD0C
S113308084180020A01800200070044034100000B0
S113309000E100E0FFFF00FF00C00440FFF8FFFE76
S11330A000600740A419002080B584B000AFF86028
S11330B0B960BB1D1A80FB689B89002B01D00823D3
S11330C020E0FEF705FFFB68BA689A60FB68BA1D4A
S11330D012889A81FB6800229A800C4BDB78DBB261
S11330E0DBB25BB2002B01DA084B5B79074B074A72
S11330F01278D2B2802149420A43D2B21A70FEF742
S1133100F7FE0023181CBD4604B080BD00600740D4
S113311080B584B000AFF860B960BB1D1A80FB684D
S11331209B8A002B01D0082316E0FEF7D1FEFB6832
S1133130BA681A61FB68BA1D12889A82FB68002279
S1133140DA81074B064A1278D2B220210A43D2B25E
S11331501A70FEF7CDFE0023181CBD4604B080BDD6
S11331600060074080B582B000AF344B1B687B60C1
S1133170334AFB1CD2781A70FB1C1B785BB2002B01
S113318028DA7B689B89002B24D07B689B682C4AB7
S11331905279D2B21A705A1C7B689A607B689B88F9
S11331A001339AB27B689A807B689A887B689B8992
S11331B09A420FD1224B224A1278D1B27F220A407E
S11331C0D2B21A707B6800229A817B689B69181CB2
S11331D000F06AF9FB1C1A78202313402AD07B687C
S11331E0DA897B689B8A9A421CD2154A7B681B69E0
S11331F0197851715A1C7B681A617B68DB89013329
S11332009AB27B68DA817B68DA897B689B8A9A4206
S113321010D17B6800229A827B689B69181C00F09D
S11332208DF907E0064B064A1278D2B220218A4370
S1133230D2B21A70BD4602B080BDC046A0180020AC
S11332400060074090B585B000AF78602B4B1B88B9
S11332509BB2002B45D03B1C0F33EFF3108072B6AA
S11332601870274B1B78DBB20133DBB2244A191CDC
S11332701170012B04D13B1C0F331A78214B1A70A7
S11332801E4B1B889BB2013B9AB21C4B1A801E4BEF
S11332901B781A1C1D49895C7A6811700133DAB2F3
S11332A0194B1A70184B1B782F2B02D9164B00227E
S11332B01A70174B1C78164B1B7841229343DAB2D1
S11332C0134B1A700E4B1B78DBB2013BDBB20C4A7A
S11332D0191C1170002B06D10A4B187880F3108842
S11332E001E00A2306E0221C4123134001D00D23F0
S11332F000E00023181CBD4605B090BDA6180020B0
S1133300E4190020781C0020A8180020AC18002024
S1133310A418002080B584B000AF021CFB1D1A70F5
S1133320304B1B889BB2302B01D10B2355E03B1C47
S11333300F33EFF3108072B618702B4B1B78DBB28F
S11333400133DBB2284A191C1170012B04D13B1C38
S11333500F331A78254B1A70224B1B889BB201330A
S11333609AB2204B1A80224B1B781A1C2149F81D53
S1133370007888540133DAB21D4B1A701C4B1B7849
S11333802F2B02D91A4B00221A701B4B1B781A1CC4
S11333902023134012D1184B1B7820221343DAB296
S11333A0154B1A70154B1A68154B1B78191C114BC9
S11333B0CB18101C191C0122FFF7AAFE0A4B1B781C
S11333C0DBB2013BDBB2084A191C1170002B03D19C
S11333D0064B187880F310880023181CBD4604B0EF
S11333E080BDC046DE180020E4190020781C0020AF
S11333F0E1180020E4180020A4180020741C002008
S1133400E018002080B500AF024B1B889BB2181C4B
S1133410BD4680BDA618002080B500AF024B1B88B6
S11334209BB2181CBD4680BDDE18002080B500AFDD
S1133430134B00221A70134B00221A70124B0022F5
S11334401A80124B00221A70114B00221A70114B71
S113345000221A80104B00221A70104B00221A709E
S11334600020FFF79BFD021C0D4B1A600C4B1A68E1
S11334700C4B101C191C0122FFF716FEBD4680BD23
S1133480A4180020A5180020A6180020A8180020C1
S1133490A9180020DE180020E0180020E118002000
S11334A0741C0020DC18002080B582B000AF786066
S11334B01B4B1B889BB22F2B19D8194B1B889BB213
S11334C001339AB2164B1A80164B1B781A1C1649F4
S11334D00878164988540133DAB2124B1A70114B2A
S11334E01B782F2B11D90F4B00221A700DE0104BB3
S11334F01B7840221343DAB20D4B1A700D4B1B7824
S113350040221343DAB20B4B1A700B4B1A68064B6A
S1133510101C191C0122FFF7C7FDBD4602B080BD77
S1133520A6180020A9180020DC180020AC180020E0
S1133530A4180020A5180020741C002080B582B0B7
S113354000AF78601B4B1B780133DAB2194B1A7049
S1133550184B1B782F2B02D9164B00221A70164BCE
S11335601B889BB2013B9AB2134B1A80124B1B88E7
S11335709BB2002B13D0114B1B7820221343DAB2D9
S11335800E4B1A700E4B1A680A4B1B78191C0D4B04
S1133590CB18101C191C0122FFF7BAFD06E0074BDB
S11335A01B7830229343DAB2044B1A70BD4602B042
S11335B080BDC046E0180020DE180020A4180020BA
S11335C0741C0020E418002080B582B000AF78603D
S11335D003F020FD031C9B687A68101C191C03F07F
S11335E09DFABD4602B080BD80B500AF024B0122FA
S11335F01A70BD4680BDC0467019002080B582B0E7
S113360000AFFB1D00221A7001F036FA031C002BD8
S113361002D0FB1D1B221A7001F036FA031C002B8A
S113362002D0FB1D1B221A70E22002F087F8E12071
S113363002F084F8FB1D1B78181CBD4602B080BD47
S113364080B500AF00200C2101F0B0FFFFF7D6FFDA
S1133650031C181CBD4680BD80B584B000AF3B1C64
S11336600F3300221A70234B181C222101F01EFD77
S1133670031C002B39D13B1C0E331E4A12781A70DE
S11336803B1C0E331A780423134003D0FFF7D8FFF2
S113369007232BE002F0F4F800200E2101F086FF4E
S11336A03B1C144A5A603B1C3A1C0E3212781A70A6
S11336B03B1C22225A703B1C5B689A1C3B1C9A6080
S11336C00D4B1B78002B04D03B1C181C012101F06E
S11336D01DFA3B1C9A683B1C5B6801331B78101C69
S11336E0191C02F089F8002300E00923181CBD46C8
S11336F004B080BD181900201419002090B58FB0B3
S113370000AF3B1C373300221A703B1C36330022B7
S11337101A703B1D00221A703B1D3A1C10325A606D
S11337203B1D22225A703B1D5B689A1C3B1D9A600C
S11337303C1C353402F03AF8031C23703B1C35332F
S11337401A78402313401ED03B1C363301221A70D2
S1133750FB1C181C02F0E4F8FB1C1B78202B04D97A
S1133760E22001F0EBFF1B2339E03B1D9A68FB1CB0
S11337701B78101C191C02F065F83B1D5B680133B3
S1133780FA1C12781A703B1C36331B78002B23D09A
S11337903B1D58683B1D5B78191C3B1D5B6801335E
S11337A01A783B1D1B783C1C373401F0E1FC031CE8
S11337B023703B1C37331B78002B0DD03B1C373355
S11337C01B78042B04D1084B181CFFF7FDFE03E003
S11337D0064B181CFFF7F8FE3B1C37331B78181CEC
S11337E0BD460FB090BDC046EC95000008960000A1
S11337F090B583B000AF4B4B1B78072B00D98AE000
S11338009A00494BD3181B689F4602F039F8454B80
S113381001221A707EE000200F2101F0C7FE02F0A1
S11338203BF8404B05221A7074E002F07BF93F4BE1
S11338301B78DBB2002B08D03C4B00221A70FFF738
S11338405DFF384B01221A7064E0394B00221A7074
S1133850344B06221A705DE0FC1DFFF7FDFE031CCD
S11338602370FB1D1B78002B03D12E4B03221A70EF
S113387050E0FB1D1B78072B03D12A4B07221A703B
S11338804CE0284B05221A7048E002F04BF9274B14
S11338901B78DBB2002B40D0244B00221A70BC1DD5
S11338A001F084FF031C2370BB1D1A7810231340FE
S11338B006D0E12001F042FF1A4B04221A7029E0DD
S11338C0184B01221A7025E0194B1B78022B19D8CA
S11338D0184B181CFFF778FE154B1B780133DAB22E
S11338E0134B1A70144B181C222101F0BFFB031C4C
S11338F0002B03D10B4B06221A700FE00F4B181C40
S1133900FFF762FE0E4B181CFFF75EFE054B01220B
S11339101A70C0466FE7C04600E0C046BD4603B01B
S113392090BDC0463C19002074A10000701900200D
S11339301519002020960000181900203096000068
S11339404896000080B582B000AF021CFB1D1A70BF
S1133950FB1D1B78181C01F0ABFF031C181CBD4693
S113396002B080BD80B500AF01F010FE0620062134
S113397001F01CFE072001F0FBFF012001F0E0FF35
S11339800020FFF7DFFF1A4B0A20191C052201F063
S113399087FE174B1020191C052201F081FE02201E
S11339A0012101F003FE702001F0F0FE012001F07E
S11339B0A3FF04202F2101F0F9FD00200F2101F0C5
S11339C0F5FDFFF71BFE01F067FF0A4B00221A709A
S11339D0094B0A4A5A60084B22225A70064B5B680C
S11339E05A1C054B9A600023181CBD4680BDC04676
S11339F06CA100003C190020401900204C19002043
S1133A0090B583B000AFFFF7F3FEFC1D0D4B181CFF
S1133A1001F042F8031C2370FB1D1B78002B0CD112
S1133A20094B1B78002B04D0064B181C002101F015
S1133A306DF8044B181C01F043F80023181CBD4614
S1133A4003B090BD401900201419002080B582B045
S1133A5000AF021CFB1D1A70FB1D1B78072B12D82C
S1133A609A000B4BD3181B689F460A4B0CE00A4B79
S1133A700AE00A4B08E00A4B06E00A4B04E00A4B52
S1133A8002E00A4B00E00A4B181CBD4602B080BDA0
S1133A9094A1000058960000609600006C96000007
S1133AA07C960000909600009C960000A89600006A
S1133AB0B496000080B582B000AF78607B685B6824
S1133AC02449254A081C111C1A1C03F069FB7B6855
S1133AD05B682249224A081C111C1A1C03F060FB73
S1133AE07B685B681F49204A081C111C1A1C03F0E0
S1133AF057FB7B685B681D491D4A081C111C1A1C76
S1133B0003F04EFB7B685B681A491B4A081C111CB6
S1133B101A1C03F045FB7B685B681849184A081CAB
S1133B20111C1A1C03F03CFB7B685B681549164AA0
S1133B30081C111C1A1C03F033FB7B685B681349D7
S1133B40134A081C111C1A1C03F02AFBBD4602B0C0
S1133B5080BDC046BC960000C4960000E0960000FC
S1133B60F096000010970000249700006C97000066
S1133B7080970000AC970000BC970000D897000025
S1133B80F097000010980000189800002C9800008E
S1133B903898000090B58DB000AF78600023FB62C8
S1133BA03DE0FB6ADBB23C1C2B34181C01F026FD03
S1133BB0031C23703A1C18321C4B101C10211A1CB5
S1133BC0FEF7E2FBFB6ADBB23A1C1832101C102130
S1133BD01A1CFEF753FE3B1C083300221A703A1CD1
S1133BE008323B1C2B331B78101C10211A1CFEF7C7
S1133BF045FE3A1C08320E4B101C10211A1CFEF70D
S1133C00E7FB7B685B68391C18313A1C0832081CD6
S1133C10111C1A1C03F0D8FAFB6A0133FB62FB6A1D
S1133C201D2BBEDDBD460DB090BDC04654980000AE
S1133C306098000080B58CB000AF78607B685B68EA
S1133C401049114A081C111C1A1C03F0BDFA0F4B31
S1133C501B78181CFFF7FAFE021C7B685B680C4992
S1133C60081C111C1A1C03F0AFFA7B685B68064A37
S1133C70101C191C02F052FF064B1B78002B0DD0B0
S1133C80054B0CE064980000609800003C1900208B
S1133C906C9800001419002074980000E74B7A68AF
S1133CA05268E749081C191C03F08EFA3B1C0F33B9
S1133CB0181C01F011FE3B1C0F331B783A1C103208
S1133CC0101C20211A1CFEF7DDFB3A1C1032DD4BC0
S1133CD0101C20211A1CFEF77BFB7B685B68DA4909
S1133CE03A1C1032081C111C1A1C03F06DFA3B1C00
S1133CF00D33181C01F0A4FE3B1C0D331B783A1C39
S1133D0010325BB2101C20211A1CFEF7CFFB3A1CA8
S1133D101032CE4B101C20211A1CFEF759FB7B6875
S1133D205B68CB493A1C1032081C111C1A1C03F0A6
S1133D304BFA3B1C0A33181C01F0C0FE3B1C0A332F
S1133D401B883A1C1032101C20211A1CFEF7C4FBDD
S1133D503A1C1032BF4B101C20211A1CFEF738FBF2
S1133D607B685B68BC493A1C1032081C111C1A1C85
S1133D7003F02AFA01F000FD031C1A1C3B1C0F334C
S1133D801A703A1C1032B54B101C20211A1CFEF775
S1133D90FBFA3B1C0F331B783A1C1032101C2021F9
S1133DA01A1CFEF76BFD3A1C1032AD4B101C20217F
S1133DB01A1CFEF70DFB3B1C0F331B781A1C402307
S1133DC0134007D03A1C1032A64B101C20211A1C99
S1133DD0FEF7FEFA3B1C0F331B781A1C20231340FA
S1133DE007D03A1C1032A04B101C20211A1CFEF7DD
S1133DF0EFFA3B1C0F331B781A1C1023134007D017
S1133E003A1C1032994B101C20211A1CFEF7E0FAC0
S1133E103B1C0F331B781A1C0E2313400E2B07D1A7
S1133E203A1C1032924B101C20211A1CFEF7D0FAB7
S1133E303B1C0F331B781A1C0E2313400C2B07D189
S1133E403A1C10328B4B101C20211A1CFEF7C0FAAE
S1133E503B1C0F331B781A1C0E2313400A2B07D16B
S1133E603A1C1032844B101C20211A1CFEF7B0FAA5
S1133E703B1C0F331B781A1C0E231340082B07D14D
S1133E803A1C10327D4B101C20211A1CFEF7A0FA9C
S1133E903B1C0F331B781A1C0E231340062B07D12F
S1133EA03A1C1032764B101C20211A1CFEF790FA93
S1133EB03B1C0F331B781A1C0E231340042B07D111
S1133EC03A1C10326F4B101C20211A1CFEF780FA8A
S1133ED03B1C0F331B781A1C0E231340022B07D1F3
S1133EE03A1C1032684B101C20211A1CFEF770FA81
S1133EF03B1C0F331B781A1C0E23134007D13A1CAA
S1133F001032624B101C20211A1CFEF761FA3B1C74
S1133F100F331B781A1C0123134007D03A1C1032AC
S1133F205B4B101C20211A1CFEF752FA3A1C10326B
S1133F30444B101C20211A1CFEF74AFA7B685B686C
S1133F4054493A1C1032081C111C1A1C03F03CF989
S1133F503B1C0F33181C01F001FE3A1C10323F4B7E
S1133F60101C20211A1CFEF70FFA3B1C0F331B7880
S1133F703A1C1032101C20211A1CFEF77FFC3A1C3C
S1133F801032374B101C20211A1CFEF721FA3B1C5F
S1133F900F331B781A1C4023134007D03A1C1032ED
S1133FA03D4B101C20211A1CFEF712FA3B1C0F3348
S1133FB01B781A1C2023134007D03A1C1032344BB0
S1133FC0101C20211A1CFEF703FA3B1C0F331B782C
S1133FD01A1C1023134007D03A1C10322F4B101C0C
S1133FE020211A1CFEF7F4F93B1C0F331B781A1C12
S1133FF00223134007D03A1C1032294B101C2021F5
S11340001A1CFEF7E5F93B1C0F331B781A1C01231D
S1134010134007D03A1C1032224B101C20211A1CCA
S1134020FEF7D6F93A1C1032064B101C20211A1C3C
S1134030FEF7CEF97B685B6836E0C0467C980000EA
S113404084980000609800008C9800009898000004
S1134050A0980000A8980000B0980000BC98000048
S1134060C0980000C4980000CC980000D4980000C8
S1134070DC980000EC980000F8980000009900001B
S11340800899000010990000189900002099000078
S113409028990000349900004099000048990000D4
S11340A0549900006099000020493A1C1032081C01
S11340B0111C1A1C03F088F83A1C0F323B1C0E33F7
S11340C0101C191C01F06CFC3B1C0F331B783A1CB0
S11340D01032101C20211A1CFEF7D4F93A1C10329D
S11340E0134B101C20211A1CFEF772F93B1C0E33D3
S11340F01B783A1C1032101C20211A1CFEF766FB98
S11341003A1C10320B4B101C20211A1CFEF760F9CC
S11341107B685B6808493A1C1032081C111C1A1C85
S113412003F052F8BD460CB080BDC0466C99000047
S11341307C990000849900009099000080B588B0B3
S113414000AFF860B9607A603B1C1F3300221A701C
S1134150FA68A14B101C191C05F025F9031C002B4F
S113416008D0FA689D4B101C191C05F01CF9031C9F
S1134170002B07D17B68181CFFF79CFCBB6801224D
S11341801A7021E1FA68964B101C191C05F00BF902
S1134190031C002B08D0FA68924B101C191C05F064
S11341A002F9031C002B07D17B68181CFFF742FDA2
S11341B0BB6801221A7007E1FA688B4B101C191CAA
S11341C005F0F1F8031C002B06D1884B01221A706C
S11341D0BB6801221A70F7E0FA68854B101C191CA1
S11341E005F0E1F8031C002B06D1804B00221A7065
S11341F0BB6801221A70E7E0FA687E4B101C191C98
S11342000D2205F0E6F8031C002B2AD1FB680E33BF
S1134210BB613A1C18323B1C1733101C191CFEF7E7
S113422069FC031C002B10D13B1C17331B78DBB239
S11342305BB2002B09DB3B1C17331B78181CFFF700
S113424081FBBB6801221A70BEE07B689B686A4AE6
S1134250101C191C02F062FC3B1C1F331B221A7039
S1134260B2E0FA68654B101C191C0B2205F0B1F87A
S1134270031C002B3ED1FB680C33BB613A1C183283
S11342803B1C1633101C191CFEF788FC031C002B66
S113429024D13B1C16331B78002B14D03B1C163343
S11342A01B785BB21A1C0A320DD03B1C16331B78E8
S11342B05BB21A1C0C3206D03B1C16331B785BB263
S11342C01A1C12320AD13B1C16331B78DBB2181CA1
S11342D001F086FBBB6801221A7075E07B689B685D
S11342E0474A101C191C02F019FC3B1C1F331B22EB
S11342F01A7069E0FA68434B101C191C0E2205F071
S113430068F8031C002B32D1FB680F33BB613A1CE5
S113431018323B1C1533101C191CFEF715FD031C29
S1134320002B18D13A1C18323B1C1733101C191CD3
S1134330FEF70AFD031C002B0DD13B1C15331A7824
S11343403B1C17331B78101C191C01F02FF9BB6898
S113435001221A7038E07B689B682B4A101C191CD8
S113436002F0DCFB3B1C1F331B221A702CE0FA68A2
S1134370264B101C191C05F016F8031C002B13D136
S1134380BB6801221A70FFF739F9031C002B1BD0FC
S11343907B689B681E4A101C191C02F0BFFB3B1C67
S11343A01F331B221A700FE0FA681A4B101C191CD9
S11343B004F0F9FF031C002B06D17B68181CFFF7DF
S11343C0E9FBBB6801221A703B1C1F331B78181CC5
S11343D0BD4608B080BDC046A0990000A899000061
S11343E0B4990000BC990000CC9900001419002075
S11343F0DC990000EC990000FC9900002C9A000064
S1134400389A0000689A0000789A00008C9A00009C
S1134410989A0000AC9A000080B500AF024B0022CD
S11344201A70BD4680BDC0461419002080B584B002
S113443000AFF860B9607A6014E0F968BA68FA23EA
S11344405B00081C111C1A1C0023FDF78DF9031CCA
S1134450012B01D0122309E0BB680133BB607B68E8
S1134460013B7B607B68002BE7D10023181CBD4611
S113447004B080BD80B584B000AFB9607A603B1CE5
S11344800F33021C1A703B1C0F331B78052B46D8C4
S11344909A00254BD3181B689F46244B1968BA68A9
S11344A07B68081C111C1A1CFFF7C0FF031C37E0B3
S11344B01F4B1968BA687B68081C111C1A1CFFF78B
S11344C0B5FF031C2CE01B4B1968BA687B68081CF9
S11344D0111C1A1CFFF7AAFF031C21E0164B1968D4
S11344E0BA687B68081C111C1A1CFFF79FFF031C89
S11344F016E0124B1968BA687B68081C111C1A1C58
S1134500FFF794FF031C0BE00D4B1968BA687B6836
S1134510081C111C1A1CFFF789FF031C00E01B2355
S1134520181CBD4604B080BDB4A10000741900205D
S1134530781900207C19002080190020841900209B
S11345408819002080B582B000AF78607B68181CA1
S1134550FDF70EFB031C9BB2181CBD4602B080BDC8
S113456080B582B000AF021CFB1D1A70FB1D1B78C6
S1134570052B34D89A001C4BD3181B689F461B4B41
S11345801B68181CFFF7DEFF031CDBB228E0184B86
S11345901B68181CFFF7D6FF031CDBB220E0154B89
S11345A01B68181CFFF7CEFF031CDBB218E0124B8C
S11345B01B68181CFFF7C6FF031CDBB210E00F4B8F
S11345C01B68181CFFF7BEFF031CDBB208E00C4B92
S11345D01B68181CFFF7B6FF031CDBB200E00023C6
S11345E0181CBD4602B080BDCCA100007419002087
S11345F0781900207C1900208019002084190020DB
S11346008819002080B584B000AF78607A683B1CBC
S11346100B33101C191C00220023FDF7CBF9031CDB
S1134620FB60FB68002B01D1002302E03B1C0B3331
S11346301B78181CBD4604B080BDC04680B582B04E
S113464000AF021CFB1D1A70FB1D1B78052B2ED816
S11346509A00194BD3181B689F46184B1B68181CEB
S1134660FFF7D0FF031C23E0154B1B68181CFFF752
S1134670C9FF031C1CE0134B1B68181CFFF7C2FF87
S1134680031C15E0104B1B68181CFFF7BBFF031C31
S11346900EE00E4B1B68181CFFF7B4FF031C07E069
S11346A00B4B1B68181CFFF7ADFF031C00E0002335
S11346B0181CBD4602B080BDE4A10000741900209E
S11346C0781900207C19002080190020841900200A
S11346D08819002080B582B000AF3A601A1CFB1D17
S11346E01870BB1D19707B1D1A70FB1D1B78012BE4
S11346F010D0022B1BD0002B26D13B6901221A704B
S1134700BB1D1B783A680020111C1A1CFFF7B2FE6F
S1134710031C1BE03B6901221A70BB1D1B783A681D
S11347200120111C1A1CFFF7A5FE031C0EE03B69B7
S113473001221A70BB1D1B783A680220111C1A1C36
S1134740FFF798FE031C01E0C0460023181CBD4679
S113475002B080BD90B593B002AF0A1CFB1D011CD2
S11347601970BB1D1A703B1C373300221A703B1C96
S11347700C330833BB633B1C3F3300221A701CE02C
S11347803C1C3634FB1D1B78181CFFF757FF031C19
S113479023703B1C36331B78002B14D0BB6B3A1CA4
S11347A0363212781A70BB6B0133BB633B1C3F3348
S11347B03A1C3F32127801321A703B1C3F331B788B
S11347C0192BDDD900E0C046214B18783C1C373446
S11347D0391C0C313B1C3F331A78BB1D1B780090ED
S11347E002200190081C222101F0C8F9031C237047
S11347F03B1C37331B78002B23D002F00BFC031C2B
S11348003B633B6B9B682A2098473B6B9B68462025
S113481098473B6B9B68412098473B6B9B684920BA
S113482098473B6B9B684C2098473B6B9B682A20BE
S113483098473B6B9B680A2098473B1C37331B788F
S113484002E03B1C37331B78181CBD4611B090BDE9
S11348508C19002080B582B000AF021CFB1D1A70B9
S1134860FB1D0420191C0122FFF704FEFB1D1B780D
S11348700A2B05D00420FFF773FE031C1A2B03D95F
S113488004200121FFF766FFBD4602B080BDC0468B
S113489080B582B000AF021CFB1D1A70FB1D052001
S11348A0191C0122FFF7E6FDFB1D1B780A2B05D01E
S11348B00520FFF755FE031C1A2B03D905200221FE
S11348C0FFF748FFBD4602B080BDC04680B582B048
S11348D000AF78600020FFF7B1FE031C1A1C7B6850
S11348E01A70BD4602B080BD80B500AF054B1B6891
S11348F0181CFFF727FE031C5A1E9341DBB2181C39
S1134900BD4680BD7419002080B500AF014B181C52
S1134910BD4680BDFCA1000090B585B000AF7860B5
S1134920184B1B683C1C0F34181CFFF76BFE031C50
S113493023703B1C0F331B78002B07D07B685B680C
S11349403A1C0F321278101C9847E9E7C0460E4B08
S11349501B683C1C0F34181CFFF754FE031C237007
S11349603B1C0F331B78002B07D07B689B683A1CD9
S11349700F321278101C9847E9E7C046BD4605B0CF
S113498090BDC046781900207C19002080B500AF86
S1134990294BFF221A70302001210022FCF7F4FD7C
S11349A0021C264B1A60254B1B68002B00D1FEE726
S11349B0302001210022FCF7E7FD021C204B1A6085
S11349C01F4B1B68002B00D1FEE730200121002281
S11349D0FCF7DAFD021C1B4B1A601A4B1B68002BF8
S11349E000D1FEE7302001210022FCF7CDFD021C9E
S11349F0154B1A60144B1B68002B00D1FEE73020C6
S1134A0001210022FCF7C0FD021C104B1A600F4B61
S1134A101B68002B00D1FEE7302001210022FCF7A7
S1134A20B3FD021C0A4B1A60094B1B68002B00D112
S1134A30FEE7BD4680BDC0468C19002074190020D5
S1134A40781900207C190020801900208419002086
S1134A508819002080B500AFFFF7DEFC00F0AAFB48
S1134A6000F066F800F0FEFC00F016FAFFF78EFF87
S1134A7001F05AFBBD4680BD80B500AF00F048FA96
S1134A80031C181CBD4680BD80B500AF00F054FA6D
S1134A90031C181CBD4680BD80B582B000AF786091
S1134AA07B6800221A707B685A687B685B78101CEC
S1134AB0191C00F01BFB031C181CBD4602B080BD72
S1134AC080B582B000AF78607B68181C00F0CEFB24
S1134AD0031C181CBD4602B080BDC04680B584B01E
S1134AE000AFF860B960111C1A1CFB1D1970BB1DC6
S1134AF01A70F868B968FB1D1A78BB1D1B7800F0A2
S1134B0015FB031C181CBD4604B080BD80B582B0E3
S1134B1000AF78600A1CFB1C1A707A68FB1C1B78B7
S1134B20101C191C00F0F0FBBD4602B080BDC0464D
S1134B3080B500AFBD4680BD80B500AF024B1B7889
S1134B40181CBD4680BDC0460CF0FF1F80B582B066
S1134B5000AF021CFB1D1A70044BFA1D12781A7068
S1134B600023181CBD4602B080BDC0460CF0FF1FD8
S1134B7080B582B000AF7860034B7A681A60002376
S1134B80181CBD4602B080BD9019002090B587B0B6
S1134B9000AFF860B960111C1A1CFB1D1970BB1D15
S1134BA01A703C1C1734FFF7C7FF031C2370FB6803
S1134BB004333A1C173212781A70FB680533BA1D95
S1134BC012781A70FB1D1B780233DAB2F868B968E0
S1134BD03B1C28331B7800F00FFB031C181CBD463C
S1134BE007B090BD80B58EB000AF78600A1CFB1C86
S1134BF01A703B1C083300221A703B1C08333A1C01
S1134C0014325A603B1C083322225A707B685A685B
S1134C103B1C373312791A703B1C08335B6804332E
S1134C20FA1C12781A703B1C08335B6805333A1C73
S1134C30373212781A707A683B1C0833101C191C1E
S1134C4000F022FB031C181CBD460EB080BDC046FC
S1134C5090B585B000AF78607B685A683B1C0F3311
S1134C6052791A703B1C0F331B78FF2B07D0FFF7C8
S1134C7063FF031C3A1C0F3212789A4246D17B68B8
S1134C805A687B685B783C1C0E34101C191C00F0BD
S1134C901BFB031C23703B1C0E331A7802231340A6
S1134CA013D07B685A687B685B78101C191C00F071
S1134CB017FB031C002B08D07B681B7801221343CD
S1134CC0DAB27B681A70002321E03B1C0E331A7899
S1134CD00123134018D0104B1B68002B16D03B1C2B
S1134CE00E331B785BB2002B07DAFFF725FF031C9A
S1134CF07A68101C191CFFF775FF074B1B687A684C
S1134D00101C9847031C02E0122300E01B23181C0C
S1134D10BD4605B090BDC0469019002080B582B054
S1134D2000AF78600A1CFB1C1A707A68FB1C1B78A5
S1134D30101C191C01F04EF8BD4602B080BDC046DF
S1134D4080B582B000AF78607B685B680A490B4A23
S1134D50081C111C1A1C02F023FA7B685B680849C2
S1134D60084A081C111C1A1C02F01AFA0023181C09
S1134D70BD4602B080BDC046BC9A0000C49A000083
S1134D80E09A0000F09A000080B58AB000AF786025
S1134D907B685B681749184A081C111C1A1C02F02E
S1134DA013FA3A1C0832154B101C20211A1CFDF76B
S1134DB0EBFAFFF7C1FE031C3A1C0832101C202139
S1134DC01A1CFDF75BFD3A1C08320B4B101C20210A
S1134DD01A1CFDF7FDFA7B685B6809493A1C083226
S1134DE0081C111C1A1C02F0EFF90023181CBD4604
S1134DF00AB080BDBC9A0000089B00000C9B000018
S1134E00109B000080B584B000AFF860B9607A6090
S1134E10FA681D4B101C191C04F0C5FA031C002B66
S1134E2008D0FA68194B101C191C04F0BCFA031CB6
S1134E30002B08D1BB6801221A707B68181CFFF78D
S1134E407FFF031C1BE0FA68114B101C191C04F0B3
S1134E50AAFA031C002B08D0FA680E4B101C191C6C
S1134E6004F0A1FA031C002B08D1BB6801221A70BC
S1134E707B68181CFFF788FF031C00E00023181C44
S1134E80BD4604B080BDC046189B0000209B0000B6
S1134E902C9B0000349B000080B500AF034BFF2225
S1134EA01A70034B00221A60BD4680BD0CF0FF1F30
S1134EB09019002080B500AFBD4680BD80B500AF1D
S1134EC0FFF7C8FDBD4680BD80B500AFFEF798FD75
S1134ED0031C181CBD4680BD80B500AFFEF742FD23
S1134EE0031C181CBD4680BD80B584B000AFF860BB
S1134EF0B9607A60F868B9687A68044B01F0A0FF79
S1134F00031C181CBD4604B080BDC0460CA20000A2
S1134F1080B500AF074B1B68181C0021FCF7DEFAB4
S1134F20031C012B01D01B2300E00023181CBD46E9
S1134F3080BDC0469419002080B500AF074B1B68A4
S1134F40181C0021FCF7CAFA031C012B01D01B23F7
S1134F5000E00023181CBD4680BDC04698190020FF
S1134F6080B588B000AFF860B960111C1A1CFB1D35
S1134F701970BB1D1A703B1C1F3300221A70FB1DD5
S1134F801B78202B01D9042368E0BB68222B01D0B5
S1134F901B2363E03B1C28331B78002B03D0314BCD
S1134FA01B68BB6102E0304B1B68BB61FB683A1CA9
S1134FB0303212781A70FB680133FA1D12781A70B5
S1134FC0BB1D1B78002B25D03B1C2C331B78002BDE
S1134FD00CD0B969FA683B1C1033081C111C1A1C4C
S1134FE00023FCF781FC031C7B610BE0B969FA68C0
S1134FF03B1C1033081C111C1A1C0123FCF774FC05
S1135000031C7B617B69012B25D03B1C1F330822C9
S11350101A7020E03B1C2C331B78002B0AD0BA6991
S1135020FB68101C191CC8220023FCF79DFB031C01
S11350307B6109E0BA69FB68101C191CC8220123B2
S1135040FCF792FB031C7B617B69012B03D03B1CA7
S11350501F3308221A703B1C1F331B78181CBD46D3
S113506008B080BD981900209419002080B582B042
S113507000AF786039603B68212B01D804230EE02F
S1135080094B1A687B68101C191C00220123FCF7C9
S11350906BFB031C012B01D1002300E00A23181C25
S11350A0BD4602B080BDC0469819002080B582B0CC
S11350B000AF786039603B68212B01D804230EE0EF
S11350C0094B1A687B68101C191C00220023FCF78A
S11350D071FC031C012B01D1002300E00A23181CDE
S11350E0BD4602B080BDC0469819002080B582B08C
S11350F000AF786039603B68212B01D804230EE0AF
S1135100094B1A687B68101C191C00220023FCF749
S113511051FC031C012B01D1002300E00A23181CBD
S1135120BD4602B080BDC0469419002080B588B049
S113513004AFF860B960111C1A1CFB1D1970BB1D6B
S11351401A70F968BA68FB1D1B78012000900120D1
S11351500190B81D00780290081C111C1A1C002331
S1135160FFF7FEFE031C181CBD4604B080BDC046FC
S113517080B588B004AFF860B960111C1A1CFB1D1F
S11351801970BB1D1A70F968BA68FB1D1B780020E2
S1135190009001200190B81D00780290081C111C99
S11351A01A1C0023FFF7DCFE031C181CBD4604B0C8
S11351B080BDC04680B500AF062022210022FCF746
S11351C0E3F9021C0A4B1A60094B1B68002B00D13F
S11351D0FEE7062022210022FCF7D6F9021C054B2B
S11351E01A60044B1B68002B00D1FEE7BD4680BD4E
S11351F0941900209819002080B584B000AFF8609D
S1135200B960111C1A1CFB1D1970BB1D1A70BB1D43
S11352101A780223134004D0FB68023381221A70E7
S113522003E0FB68023301221A700E4B1A780E4B0E
S11352301A70FB68DA1C0B4B1B78191C11700133B4
S1135240DAB2084B1A70FB1D1B780233DAB2F86825
S1135250B968BB1D1B78FFF741FC031C181CBD4635
S113526004B080BD9C1900209D19002080B582B037
S113527000AF78607B68181CFFF7EAFC031C181C5D
S1135280BD4602B080BDC04680B582B000AF786034
S113529039603B685B68023302221A703B685B68C2
S11352A0DA1C7B685B68DB7813703B685A683B6880
S11352B05B78101C191C04220023FFF70FFC031C4D
S11352C0181CBD4602B080BD80B582B000AF7860C6
S11352D039607B6802331B78181CBD4602B080BD60
S11352E080B582B000AF786039607B6803331A7888
S11352F0044B1B78D31A5A425341DBB2181CBD46E7
S113530002B080BD9D19002080B582B000AF7860E6
S11353100A1CFB1C1A707A68FB1C1B78101C191CD5
S1135320FFF7FCFCBD4602B080BDC04680B586B028
S113533000AFF860B9607A603B1C173301221A7021
S11353407B685B689A1C3B1C163312781A70FB68E6
S113535000221A70FA68BB68101C191C2822FDF779
S113536069F83B1C16331B785BB2002B0CDAF96826
S1135370BA68374B081C111C1A1CFDF729F83B1C92
S1135380173300221A700BE0F968BA68314B081C15
S1135390111C1A1CFDF71CF83B1C173300221A7051
S11353A03B1C16331A780123134017D03B1C1733C8
S11353B01B78002B06D1FA68BB68101C191C7C22D0
S11353C0FDF738F8F968BA68234B081C111C1A1C3D
S11353D0FCF7FEFF3B1C173300221A703B1C1633EC
S11353E01A780223134017D03B1C17331B78002B69
S11353F006D1FA68BB68101C191C7C22FDF71AF848
S1135400F968BA68154B081C111C1A1CFCF7E0FF5C
S11354103B1C173300221A703B1C16331A780423E2
S113542013400BD0F968BA680D4B081C111C1A1CE8
S1135430FCF7CEFF3B1C173300221A70FA68BB68D6
S1135440101C191C2922FCF7F5FFBD4606B080BDCF
S1135450409B0000489B0000509B0000589B0000AC
S11354605C9B000080B500AF034B00221A70034B15
S113547000221A70BD4680BD9C1900209D19002091
S113548080B584B000AF021CFB1D1A70C046FDF746
S1135490C3FF031C002BFAD1C046FB1D1B78181C4C
S11354A0FDF738FF031C002BF7D1C046FDF7B4FF0E
S11354B0031C002BFAD1C046FDF7A4FF031C002BEC
S11354C0FAD0C0463B1C0F33181CFDF7BBFE031C6F
S11354D0002BF7D13B1C0F331B78181CBD4604B0BE
S11354E080BDC04690B587B000AFF860B960FB1DC1
S11354F01A703B1C173300221A7016E03B1C17333A
S11355001B78BA68D4183B1C17331B78FA68D31875
S11355101B78181CFFF7B4FF031C23703B1C1733C4
S11355203A1C1732127801321A703A1C1732FB1DDA
S113553012781B789A42E1D3BD4607B090BDC046AD
S113554080B584B000AF78600A1CFB1C1A703B1C49
S11355500F3300221A700FE03B1C0F331B787A685C
S1135560D3181B78181CFFF78BFF3B1C0F333A1C16
S11355700F32127801321A703A1C0F32FB1C127867
S11355801B789A42E8D3BD4604B080BD80B500AF15
S1135590054BDB6A181C01F047FF034B1B6B181CFF
S11355A001F006FFBD4680BDA419002080B582B07D
S11355B000AF0A1CFB1D011C1970BB1D1A700E4B99
S11355C01B6B181C01F0E8FEFB1D1B782022134303
S11355D0DBB2181CFFF754FFBB1D1B78181CFFF728
S11355E04FFF054B1B6B181C01F0E2FEF020FCF78B
S11355F0A9FEBD4602B080BDA419002090B585B0B7
S113560000AF021CFB1D1A700F4B1B6B181C01F022
S1135610C3FEFB1D1B78181CFFF732FF3C1C0F3424
S11356200020FFF72DFF031C2370074B1B6B181C76
S113563001F0BEFEF020FCF785FE3B1C0F331B7807
S1135640181CBD4605B090BDA419002080B582B0D9
S113565000AF3960FB1D011C1970BB1D1A700F4B84
S11356601B6B181C01F098FEFB1D1B78181CFFF720
S113567007FF39683A68BB1D1B78081C111C1A1CEB
S1135680FFF730FF054B1B6B181C01F091FEF02057
S1135690FCF758FEBD4602B080BDC046A4190020E8
S11356A080B582B000AF3960FB1D011C1970BB1DB1
S11356B01A700F4B1B6B181C01F06EFEFB1D1B7840
S11356C020221343DBB2181CFFF7DAFE3A68BB1D35
S11356D01B78101C191CFFF733FF054B1B6B181CA0
S11356E001F066FEF020FCF72DFEBD4602B080BD41
S11356F0A419002090B583B000AF021CFB1D1A70E2
S11357000D4B1B6B181C01F047FEFC1DFB1D1B7889
S1135710181CFFF7B5FE031C2370074B1B6B181CEA
S113572001F046FEF020FCF70DFEFB1D1B78181C53
S1135730BD4603B090BDC046A419002080B582B018
S113574000AF021CFB1D1A700A4B1B6B181C01F0E6
S113575023FEFB1D1B78181CFFF792FE054B1B6BE9
S1135760181C01F025FEF020FCF7ECFDBD4602B04C
S113577080BDC046A419002080B500AFFF20FFF70C
S1135780B9FF031C181CBD4680BDC04680B582B05D
S113579000AF021CFB1D1A70FB1D1B780720191C8F
S11357A0FFF704FFBD4602B080BDC04690B583B08C
S11357B000AF104B1B6B181C01F0EEFDFC1D2720E5
S11357C0FFF75EFE031C2370FB1D1A787023134041
S11357D0DBB2181CFFF754FE064B1B6B181C01F0C0
S11357E0E7FDF020FCF7AEFDFB1D1B78181CBD4641
S11357F003B090BDA419002080B582B000AF7860DA
S11358000A1CFB1C1A70E120FFF798FF7A68FB1C46
S11358101B78A020111C1A1CFFF742FF084BDB6AFF
S1135820181C01F00DFEB4235B00181CFCF78AFD64
S1135830034BDB6A181C01F0F7FDBD4602B080BDC6
S1135840A419002080B582B000AF78600A1CFB1C4C
S11358501A700A4BDB6A181C01F0E6FD7A68FB1C1F
S11358601B786120111C1A1CFFF7F0FE034BDB6A46
S1135870181C01F0E5FDBD4602B080BDA41900204E
S113588080B500AF034BDB6A181C01F0CDFDBD46AB
S113589080BDC046A419002080B500AF034BDB6A6D
S11358A0181C01F0CDFDBD4680BDC046A4190020E2
S11358B080B582B000AF021CFB1D1A70FB1D1A7864
S11358C07F231340DBB20520191CFFF76FFE002372
S11358D0181CBD4602B080BD80B582B000AF7860B0
S11358E00520FFF78BFE031C1A1C7B681A7000232B
S11358F0181CBD4602B080BD80B582B000AF021C4A
S1135900FB1D1A70FB1D1A783F231340DBB20120E4
S1135910191CFFF74BFE0023181CBD4602B080BDC6
S113592080B582B000AF78606020FFF767FE031C8B
S11359301A1C7B681A700023181CBD4602B080BD77
S113594080B582B000AF021CFB1D1A70FB1D1B78D2
S11359503F2B01D9122306E0FB1D1B781C20191CC8
S1135960FFF724FE0023181CBD4602B080BDC046CC
S113597080B582B000AF021CFB1D1A70FB1D1B78A2
S1135980072B01D9122306E0FB1D1B781D20191CCF
S1135990FFF70CFE0023181CBD4602B080BDC046B4
S11359A090B585B000AF786039603C1C0F34082096
S11359B0FFF724FE031C23703B1C0F331B781B09C9
S11359C0DAB27B681A703B1C0F331A780F2313402A
S11359D0DAB23B681A700023181CBD4605B090BDAE
S11359E090B585B000AF021CFB1D1A703C1C0F342F
S11359F00620FFF703FE031C23703B1C0F333A1CE5
S1135A000F32127806218A431A70FB1D1B78002B73
S1135A1010D13B1C0F333A1C0F32127806210A4373
S1135A201A703B1C0F331B780620191CFFF7BEFDB0
S1135A30002300E00223181CBD4605B090BDC046FB
S1135A4090B585B000AF78603C1C0F340620FFF79A
S1135A50D5FD031C23703B1C0F331A780623134017
S1135A6003D17B68EE221A7022E03B1C0F331A78B4
S1135A7006231340022B03D17B68F4221A7017E02B
S1135A803B1C0F331A7806231340042B03D17B6885
S1135A90F6221A700CE03B1C0F331A7806231340CD
S1135AA0062B03D17B6800221A7001E0022300E078
S1135AB00023181CBD4605B090BDC04690B585B006
S1135AC000AF78603C1C0F340620FFF797FD031CE1
S1135AD023703B1C0F331A7828231340202B03D147
S1135AE07B68FA221A8018E03B1C0F331A782823AB
S1135AF0134004D17B68FA2292001A800DE03B1C0B
S1135B000F331A7828231340082B04D17B68FA2218
S1135B10D2001A8001E0022300E00023181CBD46D5
S1135B2005B090BD90B583B000AFFC1DFFF724FE17
S1135B30031C2370FB1D1A787023134008D0064BF6
S1135B40DB6A181C01F070FCFDF74EFDFFF7B2F99B
S1135B50BD4603B090BDC046A419002080B582B0F4
S1135B6000AF78601720FFF749FD031C1A1C7B68FF
S1135B701A700023181CBD4602B080BD90B587B0D2
S1135B8002AFF860B960111C1A1CFB1D1970BB1D13
S1135B901A70FB680633BA1D12781A70FB68073353
S1135BA0FA1D12781A70FB1D1B780233DAB2F868FA
S1135BB0B9683B1C20331B783C1C243424780094A3
S1135BC0FEF7E4FF031C181CBD4605B090BDC0469B
S1135BD080B58EB002AF7860081C111C1A1CFB1C27
S1135BE01870BB1C19707B1C1A70FB1C1B781A2BB9
S1135BF001D9042327E00023FB620DE0FB6A08338C
S1135C003A1C0832D3187A6812781A707B68013308
S1135C107B60FB6A0133FB62FB1C1A78FB6A9A42C5
S1135C20ECDC391C0831FB1C1A78BB1C1B78781C73
S1135C3000780090381C383000780190081C22212C
S1135C40FFF79CFF031C181CBD460CB080BDC0466A
S1135C50B0B586B002AF3A601A1CFB1D1870BB1DAC
S1135C6019707B1D1A703B1C0F3300221A70BB6A1B
S1135C70002B1AD11B2320E0BB6A1C68FB1D18787B
S1135C80BB1D19783A687B1D1B783D6A00957D6AB7
S1135C900195A047031C002B03D03B1C0F331B2290
S1135CA01A70BB6A0433BB6200E0C046BB6A1B685F
S1135CB0002BE1D13B1C0F331B78181CBD4604B0EC
S1135CC0B0BDC046F0B589B004AF3A601A1CFB1DE4
S1135CD01870BB1D19707B1D1A703B1C0E330022FB
S1135CE01A70154B1D683C1C0F34FB1D1878BB1D26
S1135CF019783A687B1D1B783E1C0E360096BE6AE6
S1135D0001960295FFF7A4FF031C23703B1C0E337E
S1135D101B78002B04D03B1C0F331B78002B03D0C3
S1135D203B1C0F331B221A703B1C0F331B78181CAF
S1135D30BD4605B0F0BDC046A019002090B589B09D
S1135D4002AF78607B685B689A1D3B1C173312783E
S1135D501A707B685A683B1C1633D2791A707B68B8
S1135D605B6808333B617B685A683B1C0F331279CC
S1135D701A703B1C173318783B1C163319783A6990
S1135D803B1C0F331B787C680094FFF79BFF031CBC
S1135D90181CBD4607B090BD80B582B000AF7860D6
S1135DA0034B7A681A600023181CBD4602B080BDFC
S1135DB0A019002080B582B000AF021CFB1D1A7030
S1135DC0FB1D1B78181CFEF7C1FE031C181CBD46E6
S1135DD002B080BD80B58EB000AF78600A1CFB1C99
S1135DE01A7001F017F9031C3B63FB1C1B78002B92
S1135DF007D03B6B5B68BA4A101C191C00F08EFE7E
S1135E0006E03B6B5B68B74A101C191C00F086FE69
S1135E103A1C0C32B44B101C20211A1CFCF7B4FAA7
S1135E207B681B783A1C0C321BB2101C20211A1CF4
S1135E30FCF706FD3B6B5B683A1C0C32101C191C0A
S1135E4000F06CFE7B681B78002B27D03B6B5B68F3
S1135E50A64A101C191C00F061FE7B681B781A1CF2
S1135E600123134006D03B6B5B68A14A101C191C2C
S1135E7000F054FE7B681B781A1C0223134006D0E2
S1135E803B6B5B689B4A101C191C00F047FE3B6B84
S1135E905B68994A101C191C00F040FE3A1C0C3235
S1135EA0964B101C20211A1CFCF76EFA7B685B7859
S1135EB03A1C0C321BB2101C20211A1CFCF7C0FC2B
S1135EC03B6B5B683A1C0C32101C191C00F026FE5C
S1135ED03B6B5B688A4A101C191C00F01FFE7B6830
S1135EE05A683B1C2F3352781A7000237B6322E0DC
S1135EF03B1C0C3300221A707B685A687B6BD318E6
S1135F001B783A1C0C32101C20211A1CFCF7B6FC1E
S1135F103A1C0C327B4B101C20211A1CFCF758FA3B
S1135F203B6B5B683A1C0C32101C191C00F0F6FD2C
S1135F307B6B01337B633B1C2F331B789A1C7B6B7D
S1135F409A42D5DC3A1C0C326F4B101C20211A1CCF
S1135F50FCF71AFA3A1C0C323B1C2F331B78101C2A
S1135F6020211A1CFCF732FC3A1C0C32674B101C23
S1135F7020211A1CFCF72CFA7B685B6802331B781F
S1135F803A1C0C32101C20211A1CFCF777FC3B6BCA
S1135F905B683A1C0C32101C191C00F0BFFD3A1C43
S1135FA00C327B68101C20211A1CFFF7BFF93B6BD5
S1135FB05B683A1C0C32101C191C00F0AFFD3A1C33
S1135FC00C32534B101C20211A1CFCF7DDF97B68A2
S1135FD05B6803331B783A1C0C32101C20211A1CFA
S1135FE0FCF74CFC3B6B5B683A1C0C32101C191C14
S1135FF000F094FD3A1C0C32464B101C20211A1C54
S1136000FCF7C2F97B685A683B1C2E3312791A706C
S11360103A1C0C323B1C2E331B78101C20211A1CFA
S1136020FCF72CFC3A1C0C323B4B101C20211A1C94
S1136030FCF7CEF97B685A683B1C2E3352791A70F0
S11360403A1C0C323B1C2E331B78101C20211A1CCA
S1136050FCF714FC3B6B5B683A1C0C32101C191CDB
S113606000F05CFD3B1C2F331B78042B2DD93A1C0C
S11360700C322A4B101C20211A1CFCF785F97B6872
S11360805B6806331B783A1C0C32101C20211A1C46
S1136090FCF7F4FB3A1C0C32214B101C20211A1C77
S11360A0FCF796F97B685B6807331B783A1C0C3263
S11360B0101C20211A1CFCF7E1FB3B6B5B683A1CAB
S11360C00C32101C191C00F029FD3B6B5B68154A4F
S11360D0101C191C00F022FDBD460EB080BDC04648
S11360E0609B00006C9B0000789B0000809B00007C
S11360F0849B00008C9B0000949B0000989B0000F4
S1136100A09B0000AC9B0000B09B0000BC9B000067
S1136110C49B0000CC9B0000D89B0000E09B0000C7
S1136120EC9B0000F49B000080B500AF044B181CEE
S1136130FEF71EFD034B00221A60BD4680BDC0461B
S11361403D5D0000A019002080B500AF024B002285
S11361501A70BD4680BDC046DC19002090B583B0DE
S113616000AFCB4B1B78012B00D180E002DC002B6D
S113617004D09AE1032B00DD97E109E1C54B5B688C
S1136180181C01F04FFA031C002B01D1012400E07C
S11361900024C04B9B68181C01F006FA031C002B5A
S11361A001D1022300E00023221C1343DCB2B94BCB
S11361B0DB68181C01F0B8F9031C002B01D104237F
S11361C000E00023221C1343DCB2B24B1B69181CF1
S11361D001F06CF9031C002B01D1082300E000231B
S11361E0221C1343DCB2AB4B5B69181C01F02AFB85
S11361F0031C002B01D1102300E00023221C1343B5
S1136200DCB2A44B9B69181C01F0DCFA031C002BC4
S113621001D1202300E00023221C1343DCB29D4B58
S1136220DB69181C01F08EFA031C002B01D14023FA
S113623000E00023221C1343DBB2DAB2964B1A703F
S1136240954B1B78002B00D12EE1944B00221A8031
S11362508F4B01221A70904B1B78181C02F056FBCE
S11362608F4B00200A211A1CFCF7BAFD1DE1894B53
S11362705B68181C01F0D6F9031C002B01D1012422
S113628000E00024834B9B68181C01F08DF9031C6B
S1136290002B01D1022300E00023221C1343DCB2B3
S11362A07C4BDB68181C01F03FF9031C002B01D167
S11362B0042300E00023221C1343DCB2754B1B694A
S11362C0181C01F0F3F8031C002B01D1082300E093
S11362D00023221C1343DCB26E4B5B69181C01F0D3
S11362E0B1FA031C002B01D1102300E00023221C6F
S11362F01343DCB2674B9B69181C01F063FA031C5F
S1136300002B01D1202300E00023221C1343DCB224
S1136310604BDB69181C01F015FA031C002B01D13A
S1136320402300E00023221C1343DAB2FB1D1A7041
S1136330594B1B78FA1D12789A421FD1574B1B8870
S113634001339AB2554B1A80544B1A88554B9A42D2
S11363500DD9524BFA2252001A804D4B03221A7067
S11363604F4B002001211A1CFCF73AFD9DE04C4BD9
S1136370002001211A1CFCF733FD96E0444B022255
S11363801A70474B002001211A1CFCF729FD8CE0F0
S1136390404B5B68181C01F045F9031C002B01D12C
S11363A0012400E000243B4B9B68181C01F0FCF81E
S11363B0031C002B01D1022300E00023221C134301
S11363C0DCB2344BDB68181C01F0AEF8031C002B64
S11363D001D1042300E00023221C1343DCB22D4B23
S11363E01B69181C01F062F8031C002B01D108235F
S11363F000E00023221C1343DCB2264B5B69181C0B
S113640001F020FA031C002B01D1102300E000232B
S1136410221C1343DCB21F4B9B69181C01F0D2F9F8
S1136420031C002B01D1202300E00023221C134372
S1136430DCB2184BDB69181C01F084F9031C002B37
S113644001D1402300E00023221C1343DAB2FB1DD8
S11364501A70FB1D1B78002B12D10D4B1B78032BDC
S113646005D10D4B1B78181C02F06CFA04E00A4BA2
S11364701B78181C02F058FA054B00221A7014E01D
S1136480074B002001211A1CFCF7AAFC0DE0C046B2
S1136490DC190020A4190020DD190020DE190020D9
S11364A05D610000F3010000C046BD4603B090BD2D
S11364B080B500AF034B1B78002B01D1FFF74EFED4
S11364C0BD4680BDDC19002080B588B000AF78607F
S11364D07B685B685149524A081C111C1A1C00F065
S11364E073FE7B685B684F4A101C191C00F016FB96
S11364F07B685B684C4A101C191C00F00FFB7B681E
S11365005B68474A101C191C00F008FBFAF7ECF909
S1136510021C131C9B009B18DB00FB61FB69181C0D
S1136520FBF7FEFD031CBB61BB69002B11D0BA69EC
S1136530FB69101C191CFAF711FF7B685B68BA69C8
S1136540101C191C00F0EAFABB69181CFBF77EFE4C
S113655006E07B689B68354A101C191C00F0DEFAC3
S11365607B685B683249334A081C111C1A1C00F012
S11365702BFE3A1C0832FA239B00101C10211A1C13
S1136580FCF746F87B685B683A1C0832101C191C3F
S113659000F0C4FA7B685B68274A101C191C00F0E1
S11365A0BDFA3B1C0833181C10210122FCF730F8FB
S11365B07B685B683A1C0832101C191C00F0AEFAA8
S11365C07B685B681D4A101C191C00F0A7FA7B68E5
S11365D05B681B49174A081C111C1A1C00F0F4FDC7
S11365E0FBF770FE031C3A1C0832101C10211A1C05
S11365F0FCF7EAF97B685B683A1C0832101C191C2A
S113660000F08CFA7B685B680E4A101C191C00F0C1
S113661085FA0023181CBD4608B080BDF89B000015
S1136620009C0000049C0000309C0000709C000052
S11366308C9C00009C9C0000A09C0000A89C000076
S1136640B09C0000BC9C000080B582B000AF7860B4
S11366507B685B680A490B4A081C111C1A1C00F071
S11366609FFD7B685B680849084A081C111C1A1CBA
S113667000F096FD0023181CBD4602B080BDC04644
S1136680F89B0000C89C0000E49C0000F49C0000FF
S113669080B584B000AFF860B9607A60FA681D4BC9
S11366A0101C191C02F07FFE031C002B08D0FA6892
S11366B0194B101C191C02F076FE031C002B08D188
S11366C0BB6801221A707B68181CFFF7BDFF031C0E
S11366D01BE0FA68114B101C191C02F064FE031C29
S11366E0002B08D0FA680E4B101C191C02F05BFE3C
S11366F0031C002B08D1BB6801221A707B68181C8C
S1136700FFF7E2FE031C00E00023181CBD4604B0A2
S113671080BDC046189D0000209D00002C9D0000F7
S1136720349D000090B585B000AF021CFB1D1A70AB
S11367303B1C0F33EFF3108072B61870FB1D1B78EF
S1136740DB08DBB21A1C0C49CB5CD9B2FB1D1878F0
S1136750072303408020041C1C41231CDBB20B4391
S1136760DBB2D9B2044B99543B1C0F33187880F335
S11367701088BD4605B090BDE019002080B582B0F8
S113678000AF021CFB1D1A70FB1D1B78DB08DBB27B
S1136790094AD35CDBB2FA1D117807220A40802132
S11367A0081C1041021CD2B21340DBB2DBB2181C2D
S11367B0BD4602B080BDC046E019002090B583B04C
S11367C000AFBB1DEFF3108072B61870FB1D0022E2
S11367D01A7025E0FB1D1B78181CFFF7CFFF031C64
S11367E0002B18D0FB1D1B78DB08DBB21A1C1649E2
S11367F0CB5CDBB2F91D0878072101408020041C22
S11368000C41211CC9B2C943C9B20B40DBB2D9B295
S11368100D4B995408E0FB1DFA1D127801321A70D1
S1136820FB1D1B78062BD5D9BB1D187880F3108867
S1136830FB1D1B78072B04D0FB1D1B78181C02F0D2
S11368408FF8BD4603B090BDE019002080B500AFBD
S1136850024B00221A70BD4680BDC046E0190020DC
S113686080B500AF02F04EF8BD4680BD80B500AFE4
S1136870FFBEBD4680BDC04680B500AF4D4A4E49FF
S11368804E4BD1504E4A88235B010021D1504C4AD3
S11368904C4BC0218902D150494A49494A4BCB58F3
S11368A0F02149011943484BD150484B9B78DBB246
S11368B01A1C0823134007D0444B444A9278D2B29E
S11368C008210A43D2B29A703D4A3E4B4049D15006
S11368D03B4A3B493F4BCB588021490219433D4B2E
S11368E0D150374B364A1268C02109030A431A6053
S11368F0334A3349374BC958374B0B40802149043D
S11369001943344BD150354B344A916C344A0A40C4
S11369109A64324B314AD16C314A0A40DA64314BC1
S113692024225A70304B80221A702E4B9A221A70ED
S11369302C4B2C4AD278D1B21F220A40D2B2DA7040
S1136940284B01221A71274B00225A71C046254B4D
S11369509B79DBB21A1C10231340F8D1C046214B9B
S11369609B79DBB21A1C0C231340082BF7D11D4B67
S113697040225A71C0461B4B9B79DBB21A1C0C2374
S11369801340082BF7D1C046164B9B79DBB21A1C77
S113699040231340F8D0134B1A221A70C046114BEF
S11369A09B79DBB21A1C0C2313400C2BF7D1BD4688
S11369B080BDC04600E000E000000000080D0000BB
S11369C000700440441000003810000000D007405C
S11369D00000011004100000FFFFFFFC00900440C1
S11369E0FFF8FFFE004006400050064080B500AFAF
S11369F072B6424B414A5279D2B21F218A43D2B273
S1136A005A713E4B3D4A1279D2B207218A43D2B21F
S1136A101A713B4B3A4A1278D2B2D2B273218A43EA
S1136A20D2B250210A43D2B2D2B21A70344B344A91
S1136A305278D2B2D2B263218A43D2B240210A43FD
S1136A40D2B2D2B25A702E4B2D4A9278D2B21921B8
S1136A508A43D2B29A702B4B00221A702A4B2A4ACC
S1136A60116D2A4A0A40E021C9000A431A65284ADE
S1136A702749C1239B00C958264B1940C1239B00B9
S1136A80D15001F0F7FB00F029FCFBF7F1F9FCF71A
S1136A9061FA002000F09CFD002000F059FD002068
S1136AA000F018FD002000F0D7FC002000F09EFE4E
S1136AB0002000F05BFE002000F018FEFFF744FB0E
S1136AC0002000F0D3FE144B1B6A181C00F002FFD8
S1136AD0002000F0BBFD104B5B6A181C00F0EAFDBF
S1136AE0FFF7B4FEFCF7A2FC002000F06DFC0020D0
S1136AF000F022FC01F0A2FDBD4680BD00F007407D
S1136B0000D0074000E0074000900440FFF8FFFE7B
S1136B1000E100E0FFFF00FFA419002080B582B06F
S1136B2000AF7860396007E07B681A787B680133CE
S1136B307B603B68101C98477B681B78002BF3D163
S1136B40BD4602B080BDC04680B584B000AFF860D9
S1136B50B9607A60FA683C4B101C191C02F023FCE3
S1136B60031C002B08D0FA68384B101C191C02F0C7
S1136B701AFC031C002B47D17B685B68344A101C49
S1136B80191CFFF7CBFF7B685B68324A101C191C89
S1136B90FFF7C4FF7B685B682D4A101C191CFFF7C4
S1136BA0BDFF7B685B682C4A101C191CFFF7B6FFFD
S1136BB07B685B68264A101C191CFFF7AFFF7B68D3
S1136BC05B68244A101C191CFFF7A8FF7B685B68EC
S1136BD01F4A101C191CFFF7A1FF7B685B681F4943
S1136BE01F4A081C111C1A1C00F0DAFA7B685B6847
S1136BF01C491D4A081C111C1A1C00F0D1FABB6860
S1136C0001221A7000231BE0FA68184B101C191C8F
S1136C1002F0C9FB031C002B08D0FA68144B101CAB
S1136C20191C02F0C0FB031C002B08D1BB68012215
S1136C301A707B68181C00F06FF8031C00E0002336
S1136C40181CBD4604B080BD449D00004C9D00004E
S1136C50589D00005C9D00009C9D0000A89D0000C4
S1136C60B09D0000CC9D0000DC9D0000009E000053
S1136C70089E000080B582B000AF78607B685B68D6
S1136C80034A101C191CFFF749FFBD4602B080BD22
S1136C90149E000080B586B000AFF860B9607A60D9
S1136CA07B68DB689847031C002B2FD000E0C046AC
S1136CB03B1C173300221A707B681B683A1C17327E
S1136CC0101C98473B1C17331B78002B18D03B1C17
S1136CD017331A78FB681A70FB680133FB60BB68D2
S1136CE0013BBB603B1C17331B780D2B09D03B1CAD
S1136CF017331B780A2B04D0BB68012BD7D800E0CC
S1136D00C046FB6800221A70012300E00023181C0F
S1136D10BD4606B080BDC04680B582B000AF786085
S1136D207B685B68214A101C191CFFF7F7FE7B681F
S1136D305B681F4A101C191CFFF7F0FE7B685B6838
S1136D401C4A101C191CFFF7E9FE7B685B68184A93
S1136D50101C191CFFF7E2FE7B685B68134A101CC9
S1136D60191CFFF7DBFE7B685B681349134A081C98
S1136D70111C1A1C00F028FA7B685B68104A101C6E
S1136D80191CFFF7CBFE7B685B680E4A101C191CAC
S1136D90FFF7C4FE7B685B68044A101C191CFFF7EC
S1136DA0BDFE0023181CBD4602B080BD589D0000E6
S1136DB05C9D00001C9E0000309E00003C9E000074
S1136DC0489E00004C9E000080B582B000AF786001
S1136DD039603B689B68154A101C191CFFF79EFE1E
S1136DE03B689B687A68101C191CFFF797FE3B6888
S1136DF09B680F4A101C191CFFF790FE3B689B68A8
S1136E000C4A101C191CFFF789FE3B689B680A4A50
S1136E10101C191CFFF782FE3B689B68074A101C74
S1136E20191CFFF77BFEBD4602B080BD589E0000D2
S1136E30589D0000789E0000449D0000849E000040
S1136E4080B586B000AFF860B9607A603B603B1CE7
S1136E50173300221A703B68002B12D11B2318E051
S1136E603B681B68F868B9687A689847031C002B6C
S1136E7003D03B1C17331B221A703B6804333B605E
S1136E8000E0C0463B681B68002BE9D13B1C17336C
S1136E901B78181CBD4606B080BDC04690B58FB0A7
S1136EA000AFF860B9607A603B1C373300221A7077
S1136EB0FB681B78002B01D10023A6E03B1C323376
S1136EC000221A70FB681B78233B5A425341DAB202
S1136ED03B1C33331A703B1C33331B78002B02D01A
S1136EE0FB680133FB603B1C353300221A703B1CEA
S1136EF0343300221A703B1C363300221A7000E02F
S1136F00C0463B1C36331B781E2B04D93B1C37333D
S1136F101B221A706DE03B1C36331B78FA6811781B
S1136F203A1C1032D154FB680133FB603B1C3633EE
S1136F303A1C3632127801321A703B1C36331B78F5
S1136F40013B3A1C1032D35C3B2B0CD13B1C363337
S1136F501B78013B3A1C10320021D1543B1C3533C1
S1136F6001221A7010E03B1C36331B78013B3A1C9B
S1136F701032D35C002B07D13B1C353301221A702D
S1136F803B1C343301221A703B1C35331B78002B15
S1136F9029D03C1C3734381C1030391C3231BA68C3
S1136FA07B68FFF74DFF031C23703B1C32331B78B7
S1136FB0002B04D03B1C37331B78002B0BD03A1C1E
S1136FC01032BB68101C191CFFF7FEFE3B1C373344
S1136FD01B221A700DE03B1C353300221A703B1C37
S1136FE0363300221A703B1C34331B78002B87D0B5
S1136FF0C0463B1C33331B78002B03D1BB68181CE1
S1137000FFF738FE3B1C37331B78181CBD460FB006
S113701090BDC04680B500AF024B1B68181CBD462E
S113702080BDC04610F0FF1F90B587B000AFF86078
S1137030B9607A603B603B1C173300221A70FB680E
S1137040181C02F0BEF9031C3B61FA683B69D118B5
S1137050BA683B69D21A7B68081C111C1A1CFFF71A
S113706019FE031C002B54D0FB68181C02F0A9F96C
S1137070031C3B613B69002B01D11B234CE03B69A2
S1137080012B0AD1FB681B780A2B03D0FB681B7801
S11370900D2B02D1FB6800221A70BB685A1E3B6993
S11370A09A4213D83C1C1734F9687A683B68081C68
S11370B0111C1A1CFFF7F2FE031C2370FB6800224C
S11370C01A703B1C173304221A7022E03B69013BFF
S11370D0FA68D3181B780A2B06D03B69013BFA687F
S11370E0D3181B780D2B14D13B69013BFA68D318D4
S11370F000221A703C1C1734F9687A683B68081C33
S1137100111C1A1CFFF7CAFE031C2370FB68002223
S11371101A703B1C17331B78181CBD4607B090BD72
S113712080B584B000AFF860B960111C1A1CFB1D57
S11371301970BB1D1A700CE0FB681A78FB680133E8
S1137140FB60BB69101C9847BB1DBA1D1278013A3D
S11371501A70FB681B78002B0CD0BB1D1B78002B0E
S1137160EAD107E0BB6920209847BB1DBA1D1278FD
S1137170013A1A70BB1D1B78002BF3D1FB1D1A7842
S1137180BB69101C9847BB6920209847BA68BB6943
S1137190101C191CFFF7C2FCBD4604B080BDC046DC
S11371A080B586B002AFF860B9607A60FA68BB68EF
S11371B079680091101C191C3B221A23FFF7B0FFB9
S11371C0BD4604B080BDC04680B586B002AFF8604D
S11371D0B9607A60FA68BB6879680091101C191C60
S11371E03A220D23FFF79CFFBD4604B080BDC04684
S11371F090B585B000AF78600F4B1A6801235B42ED
S1137200101C191CFAF77EFA3C1C0F347B68181CFE
S113721000F03AFF031C23703B1C0F331B780A2B2E
S113722002D17B6800221A70034B1B68181CFAF702
S11372303DFABD4605B090BDE819002090B585B073
S113724000AF021CFB1D1A70124B1A6801235B422B
S1137250101C191CFAF756FA3C1C0F34FB1D1B7842
S1137260181C00F085FF031C23703B1C0F331B7894
S11372700B2B02D16420F9F731FA3B1C0F331B7836
S11372800B2BE9D0034B1B68181CFAF70FFABD4609
S113729005B090BDE819002080B582B000AF0E4B58
S11372A01A6801235B42101C191CFAF72BFA00F030
S11372B0D7FF031C5A1E9341DBB21A1CFB1D1A7024
S11372C0054B1B68181CFAF7F1F9FB1D1B78181CF9
S11372D0BD4602B080BDC046E819002080B582B02A
S11372E000AFF9F77FFF031C013B5A1E9341DAB24A
S11372F0FB1D1A70FB1D1B78002B04D1BB1DEFF383
S1137300108072B618700420FAF784F9021C094B35
S11373101A60FB1D1B78002B03D1BB1D187880F36A
S11373201088044B1B68002B00D1FEE7BD4602B059
S113733080BDC046E819002080B584B000AF7860F5
S1137340104BFB60FB687A681A600F4B0E4A526957
S113735001210A435A610C4B0B4A126801210A436A
S11373601A600A4B094A1168094A0A4080214900F7
S11373700A431A60074BFA681A63FB68181CBD4677
S113738004B080BDEC190020C0F00F4000C00440E0
S1137390FFF8FFFEA419002080B582B000AF78602A
S11373A0024B01229A60BD4602B080BDC0F00FF8C6
S11373B080B582B000AF7860024B01225A60BD46AE
S11373C002B080BDC0F00FF880B584B000AF786023
S11373D0104BFB60FB687A681A600F4B0E4A5269C7
S11373E020210A435A610C4B0B4A126820218A431C
S11373F01A600A4B094A5169094A0A408021490026
S11374000A435A61074BFA68DA62FB68181CBD46E6
S113741004B080BDF0190020C0F00F4000C004404B
S1137420FFF8FFFEA419002080B582B000AF786099
S1137430024B20229A60BD4602B080BDC0F00FF816
S113744080B582B000AF7860024B20225A60BD46FE
S113745002B080BDC0F00FF880B584B000AF786092
S11374600D4BFB60FB687A681A600C4B0B4A52693F
S113747020218A435A610A4B094A5169094A0A4040
S1137480802149000A435A61074BFA681A61FB6874
S1137490181CBD4604B080BDF419002000F00F4054
S11374A000900440FFF8FFFEA419002080B584B0CA
S11374B000AF7860064B1A6920231340FB60FB6819
S11374C05A1E9341DBB2181CBD4604B080BDC046B1
S11374D000F00FF880B584B000AF78600D4BFB600E
S11374E0FB687A681A600C4B0B4A526910218A4374
S11374F05A610A4B094A1169094A0A408021490024
S11375000A431A61074BFA68DA60FB68181CBD4627
S113751004B080BDF819002000F00F400090044032
S1137520FFF8FFFEA419002080B584B000AF786096
S1137530064B1A6910231340FB60FB685A1E9341E3
S1137540DBB2181CBD4604B080BDC04600F00FF885
S113755080B584B000AF78600D4BFB60FB687A683F
S11375601A600C4B0B4A51690B4A0A405A610B4B87
S11375700A4A116B0A4A0A40802149000A431A63E5
S1137580084BFA689A60FB68181CBD4604B080BDBD
S1137590FC19002000F00F40FFEFFFFF00900440B3
S11375A0FFF8FFFEA419002080B584B000AF786016
S11375B0064B1A6980235B011340FB60FB685A1E6B
S11375C09341DBB2181CBD4604B080BD00F00FF837
S11375D080B584B000AF78600D4BFB60FB687A68BF
S11375E01A600C4B0B4A526910218A435A610A4BA8
S11375F0094A1169094A0A40802149000A431A616B
S1137600074BFA685A60FB68181CBD4604B080BD7D
S1137610001A0020C0F00F4000C00440FFF8FFFE35
S1137620A419002080B584B000AF7860064B1A69B5
S113763010231340FB60FB685A1E9341DBB2181CF5
S1137640BD4604B080BDC046C0F00FF880B584B01C
S113765000AF7860114BFB60FB687A681A60104BCE
S11376600F4A5269802109030A435A610C4B0C4AA0
S113767011680C4A0A401A600B4B0B4AD16C0B4A36
S11376800A40802149000A43DA64094BFA685A62C5
S1137690FB68181CBD4604B080BDC046041A002017
S11376A040F00F40FFFFF7FF00A00440FFF8FFFE8B
S11376B0A419002080B582B000AF7860034B80220B
S11376C012035A60BD4602B080BDC04640F00FF8B8
S11376D080B582B000AF7860034B80221203DA6079
S11376E0BD4602B080BDC04640F00FF880B584B0FE
S11376F000AF78600D4BFB60FB687A681A600C4B36
S11377000B4A51690B4A0A405A610B4B0A4A516BA6
S11377100A4A0A40802149000A435A63084BFA681E
S1137720DA61FB68181CBD4604B080BD081A00204D
S113773000F00F40FFDFFFFF00900440FFF8FFFE62
S1137740A419002080B584B000AF7860064B1A6994
S113775080239B011340FB60FB685A1E9341DBB2FC
S1137760181CBD4604B080BD00F00FF880B584B08D
S113777000AF78600D4BFB60FB687A681A600C4BB5
S11377800B4A51690B4A0A405A610B4B0A4A516A27
S11377900A4A0A40802149000A435A62084BFA689F
S11377A09A61FB68181CBD4604B080BD0C1A002009
S11377B080F00F40FFFDFFFF00B00440FFF8FFFE24
S11377C0A419002080B584B000AF7860064B1A6914
S11377D080239B001340FB60FB685A1E9341DBB27D
S11377E0181CBD4604B080BD80F00FF880B584B08D
S11377F000AF78600D4BFB60FB687A681A600C4B35
S11378000B4A51690B4A0A405A610B4B0A4A116AE6
S11378100A4A0A40802149000A431A62084BFA685E
S11378205A61FB68181CBD4604B080BD101A0020C4
S113783080F00F40FFFEFFFF00B00440FFF8FFFEA2
S1137840A419002080B584B000AF7860064B1A6993
S113785080235B001340FB60FB685A1E9341DBB23C
S1137860181CBD4604B080BD80F00FF880B584B00C
S113787000AF7860114BFB60FB687A681A60104BAC
S11378800F4A52698021C9020A435A610C4B0C4ABF
S113789011680C4A0A401A600B4B0B4A916C0B4A54
S11378A00A40802149000A439A64094BFA681A6223
S11378B0FB68181CBD4604B080BDC046141A0020E5
S11378C040F00F40FFFFFBFF00A00440FFF8FFFE65
S11378D0A419002080B582B000AF7860034B8022E9
S11378E0D2025A60BD4602B080BDC04640F00FF8D7
S11378F080B582B000AF7860034B8022D202DA6098
S1137900BD4602B080BDC04640F00FF880B584B0DB
S113791000AF7860274BFB60FB687A685A60264B9F
S1137920FA681A60FB6800221A70FB6800229A70D9
S1137930224A2249224BCB58802109051943204B66
S1137940D150204A1F49C3239B00CB581B021B0A5A
S1137950802109061943C3239B00D150194B194AAE
S11379601268802109020A431A60174B164A1168EB
S1137970164A0A401A60144B134A5168134A0A40C3
S11379805A60134B1E229A60114B114AD2681F2170
S11379908A4307210A43DA600D4B00221A620C4B1A
S11379A040225A620B4BFA685A63FB68181CBD46A6
S11379B004B080BD181A0020201A00200070044072
S11379C03C10000000E100E000A00440FFF8FFFECE
S11379D000B00340A419002080B582B000AF7860E5
S11379E00D4B1A6A8023134001D0082310E00A4B80
S11379F0094A526A08218A435A62074B064A126AA4
S1137A0040218A431A62044B7A6852781A60002330
S1137A10181CBD4602B080BD00B0034080B586B0DE
S1137A2000AFF860B960FB1D1A70FB687B61FB1D39
S1137A301B78012B03D8FB1D1B78002B01D1962347
S1137A401AE00F4B1A6A8023134001D0082313E075
S1137A507B69FA1D12781A70BB681B78012B01D957
S1137A60822309E0BB681B78064AD35C4022134397
S1137A70DAB27B695A700023181CBD4606B080BD7B
S1137A8000B0034028A2000080B584B000AF786045
S1137A9039603B68BB603B1C0F3300221A7015E051
S1137AA03B1C0F331B785B00BA68D3180D4A391C92
S1137AB00F310978043189008A5892B21A803B1C2C
S1137AC00F333A1C0F32127801321A707B681B781C
S1137AD03A1C0F3212789A42E2D30023181CBD4696
S1137AE004B080BD00B0034080B584B000AF7860BE
S1137AF02A4B5A6A4023134001D01B234AE0274BE8
S1137B00DB6CFB60254B9B6CFA68D318FB60234B42
S1137B105B6CFA68D318FB60204B1B6CFA68D318B3
S1137B20FB601E4BDB6BFA68D318FB601B4B9B6B33
S1137B30FA68D318FB60FB685B08802212021343C7
S1137B40FB60164BFA68DA62144BDB6EFB60134B76
S1137B509B6EFA68D318FB60104B5B6EFA68D318FF
S1137B60FB600E4B1B6EFA68D318FB600B4BDB6D8E
S1137B70FA68D318FB60094B9B6DFA68D318FB6055
S1137B80FB685B08802212021343FB60034BFA6814
S1137B901A630023181CBD4604B080BD00B0034026
S1137BA080B582B000AF084B1B687B607B68012204
S1137BB09A707B685B68181C00F0E6FC034B1B6939
S1137BC0BD4602B080BDC046201A002000B003406C
S1137BD080B584B000AF7860634BFB60FB68002223
S1137BE01A81FB6800221A82FB680022DA60FB68B3
S1137BF000225A82FB6800221A83FB6800225A6121
S1137C00FB687A68DA61594BFA681A60584A58492D
S1137C10584BCB588021C9001943564BD150564B71
S1137C20554A5168554A0A40802189000A435A60DE
S1137C30514B514A9168514A0A40802189000A43B4
S1137C409A604F4A4E49C3239B00CB58FF218B4374
S1137C5080211943C3239B00D150494B484A1268E1
S1137C60802149010A431A60464B464AD278D2B26F
S1137C7008218A43D2B2DA70424B424AD278D2B255
S1137C8004218A43D2B2DA70FB6800221A80FB68AE
S1137C9000225A603B4B00229A703A4B00229A71A0
S1137CA0384B00229A72374B00225A71304A3049BD
S1137CB0354BC958354B0B408021C9041943324B0D
S1137CC0D150304B2F4A1278D2B2D2B21F218A43FC
S1137CD0D2B201210A43D2B2D2B21A70294B39224C
S1137CE05A70284B274A927AD2B2D2B21F218A43C1
S1137CF0D2B203210A43D2B2D2B29A72214B214AA0
S1137D00D27AD2B2D2B202210A43D2B2D2B2DA7257
S1137D101C4B1C4AD278D2B2D2B208210A43D2B246
S1137D20D2B2DA70174B174AD278D2B2D2B2042147
S1137D300A43D2B2D2B2DA70124B124AD278D2B219
S1137D4020210A43D2B2DA700E4B0E4A9279D2B293
S1137D500F210A43D2B29A710D4BFA681A60FB687C
S1137D60181CBD4604B080BD241A0020441A00200B
S1137D70007004403410000000900440FFF8FFFE3F
S1137D8000E100E000A0064004100000FFFFFFF344
S1137D90A419002080B586B000AFF860B960BB1D9F
S1137DA01A80FB687B61BB1D1B88002B01D18423D7
S1137DB014E07B691B8A002B01D008230EE0FAF73C
S1137DC087F87B69BA68DA607B69BA1D12881A82FF
S1137DD07B6900221A81FAF78BF80023181CBD4630
S1137DE006B080BD80B586B000AFF860B960BB1D39
S1137DF01A80FB687B61BB1D1B88002B01D1842387
S1137E0029E07B691B8B002B01D0082323E0FAF7C0
S1137E105FF87B69BA685A617B69BA1D12881A8354
S1137E207B6900225A827B691B88012213439AB220
S1137E307B691A800A4B0A4AD278D2B2802149421D
S1137E400A43D2B2DA70064B054A9279D2B29A71D9
S1137E50FAF74EF80023181CBD4606B080BDC04694
S1137E6000A0064090B583B000AF7860124BDB7978
S1137E70DBB21C1C7B681B8A002B1AD07B68DB6876
S1137E80E2B21A705A1C7B68DA607B681B89013382
S1137E909AB27B681A817B681A897B681B8A9A422A
S1137EA007D17B6800221A827B68DB69181C00F00A
S1137EB013FABD4603B090BD00A0064080B582B061
S1137EC000AF78607B685A8A7B681B8B9A421CD20D
S1137ED0194A7B685B691978D1715A1C7B685A61AD
S1137EE07B685B8A01339AB27B685A827B685A8AC0
S1137EF07B681B8B9A421CD17B6800221A837B68A7
S1137F00DB69181C00F028FA13E00B4B0A4AD278FC
S1137F10D1B27F220A40D2B2DA70074B064A927974
S1137F20D2B29A717B681B88012293439AB27B6810
S1137F301A80BD4602B080BD00A00640F0B5474699
S1137F4080B482B000AF3A4B1B687B60394B1B791D
S1137F50DBB21C1C00250026221C0F2313404BD02F
S1137F60344B0F221A71334BDB79DBB29846221C57
S1137F700223134013D0221C202313400CD042466A
S1137F80002A09D1731CDEB27B681B8802221343CA
S1137F909AB27B681A8002E004232B439DB2221C10
S1137FA00823134002D001232B439DB2221C01233A
S1137FB0134002D002232B439DB2221C04231340FE
S1137FC002D008232B439DB27B685A682B1C1A43AA
S1137FD07B685A602023221C9A43131C9CB2002EF7
S1137FE005D07B68DB69181C00F042FA04E07B686A
S1137FF0DB69181C00F0F4F9221C2023134003D081
S11380007B68181CFFF72EFF7B681B881A1C012352
S1138010134007D0221C8023134003D07B68181C14
S1138020FFF74CFFBD4602B004BC9046F0BDC0460D
S1138030441A002000A0064080B584B000AF7860E8
S113804039607B68FB60F9F743FFFB685A683B685B
S11380501A60FB6800225A60F9F74AFF0023181CD3
S1138060BD4604B080BDC04680B500AF044B1A685D
S1138070044B101C191C0122FFF78CFEBD4680BD69
S11380807C1C0020801A002080B584B000AF78608A
S11380903B1C0F3300221A702D4B1B88002B4ED033
S11380A03B1C0E33EFF3108072B61870294B1B780B
S11380B0DBB20133DBB2274A191C1170012B04D146
S11380C03B1C0E331A78244B1A70214B1B88013B3E
S11380D09AB21F4B1A80214B1B881A1C2049895CB9
S11380E07A68117001339AB21C4B1A801B4B1B889F
S11380F02F2B02D9194B00221A801A4B1B881A1CE9
S1138100194B134001D0192300E000233A1C0F320D
S11381101370144B1A88154B13409AB2114B1A80E2
S11381200C4B1B78DBB2013BDBB20A4A191C117001
S1138130002B06D1084B187880F3108801E00A233D
S113814002E03B1C0F331B78181CBD4604B080BDF5
S11381504A1A0020E4190020781C00204C1A002040
S1138160501A0020481A002041080000B6F7FFFF0B
S113817080B584B000AF021CFB1D1A70304B1A8806
S113818080235B009A4201D10B2354E03B1C0F3344
S1138190EFF3108072B618702A4B1B78DBB20133F0
S11381A0DBB2284A191C1170012B04D13B1C0F337C
S11381B01A78254B1A70224B1B8801339AB2204B34
S11381C01A80224B1B881A1C2149F81D00788854F8
S11381D001339AB21D4B1A801C4B1B88FF2B02D90A
S11381E01A4B00221A801B4B1B881A1C2023134095
S11381F012D1184B1B88202213439AB2154B1A80B4
S1138200154B1A68154B1B88191C114BCB18101CE5
S1138210191C0122FFF7E6FD0A4B1B78DBB2013B78
S1138220DBB2084A191C1170002B03D1064B1878D5
S113823080F310880023181CBD4604B080BDC046DE
S1138240821A0020E4190020781C0020861A0020DD
S1138250881A0020481A00207C1C0020841A002060
S113826080B500AF024B1B88181CBD4680BDC046BC
S11382704A1A002080B500AF0F4B00221A800F4B22
S113828000221A800E4B00221A800E4B00221A8004
S11382900D4B00221A800D4B00221A800C4B002239
S11382A01A800020FFF794FC021C0A4B1A60FFF7A7
S11382B0DBFEBD4680BDC046481A00204A1A002095
S11382C04C1A00204E1A0020821A0020841A002022
S11382D0861A00207C1C002080B582B000AF786034
S11382E0174B1B882F2B18D8154B1B8801339AB2B8
S11382F0134B1A80134B1B881A1C13490878134913
S1138300885401339AB20F4B1A800E4B1B882F2BC3
S11383100AD90C4B00221A8006E00D4B1B88402220
S113832013439AB20A4B1A800A4B1A68064B101C64
S1138330191C0122FFF72EFDBD4602B080BDC046C8
S11383404A1A00204E1A0020801A0020501A0020D9
S1138350481A00207C1C002080B582B000AF7860F1
S11383601A4B1B8801339AB2184B1A80174B1B887F
S1138370FF2B02D9154B00221A80154B1B88013B99
S11383809AB2134B1A80124B1B88002B13D0114B3B
S11383901B88202213439AB20E4B1A800E4B1A6884
S11383A00A4B1B88191C0D4BCB18101C191C0122DD
S11383B0FFF718FD06E0074B1A88DF2313409AB233
S11383C0044B1A80BD4602B080BDC046841A00200A
S11383D0821A0020481A00207C1C0020881A0020E1
S11383E080B584B000AF78601F4B1A683B1C0C3317
S11383F0101C191CFFF720FEFB68002B31D0FA6813
S11384000223134001D0042300E00023174A1288FA
S113841013439AB2154B1A80FA680823134001D00B
S1138420802300E00023114A128813439AB20F4BB1
S11384301A80FB689AB2012313409AB20B4B1B8833
S113844013439AB2094B1A80FA680423134001D0EB
S1138450022300E00023054A128813439AB2034B17
S11384601A80BD4604B080BD7C1C0020481A002040
S113847080B582B000AF7860044B1B88022213439E
S11384809AB2024B1A80BD4602B080BD481A002041
S113849080B500AF034B00221A80024B00225A80A1
S11384A0BD4680BD801C002080B500AF0F4B1B78FB
S11384B0DBB2002B17D00E4B00221A700D4B00229A
S11384C01A70FFF7E5FF0C4B00221A700B4B1A6869
S11384D0094B101C191C0122FFF7A0FA074B1B685B
S11384E0181CFFF779FABD4680BDC046891B0020E1
S11384F0901B0020881B00208C1B0020841C002063
S113850080B582B000AF021CFB1D1A700D4B1B78A6
S1138510DBB2002B01D008230FE00A4B01221A70B2
S1138520FFF7C2FFFB1D1B78002B05D0C046054B8F
S11385301B78DBB2012BFAD00023181CBD4602B015
S113854080BDC046891B002080B582B000AF786032
S11385500B4B1B78DBB2002B01D109230BE0094B39
S11385601B889AB27B681A807B680233054A52885A
S113857092B21A800023181CBD4602B080BDC046CA
S1138580901B0020801C002080B582B000AF786072
S1138590244B1B78DBB2042B0AD1234B1B68181C19
S11385A0FFF7A2FA1F4B00221A7000F001FA35E01F
S11385B01D4B1A681D4B1B78DBB259001C4BCB18A2
S11385C0101C191CFFF760FA184B1B78DBB201333F
S11385D0DAB2164B1A70154B1B78DBB2022B0BD197
S11385E0124B00221A70134B01221A7000F0DCF9AE
S11385F00C4B00221A7011E00C4B1B78DAB20E4BB4
S11386001A70094B1A680C4B101C191C0122FFF735
S113861005FA054B1B68181CFFF7DEF9BD4602B0CE
S113862080BDC046891B0020841C0020881B0020BC
S1138630801C0020901B00208C1B002080B500AF04
S1138640064B00221A70064B00221A700020FFF716
S11386505DF9021C034B1A60BD4680BD901B0020CF
S1138660891B0020841C002080B500AF054A064BFE
S1138670D31A054A101C00211A1C00F08EFEBD46B8
S113868080BDC046881C002018F0FF1F00F07CFF4E
S1138690FEF7F2F8FFF7E8FF00F04EFF00F0EAFE05
S11386A000F080FF044B0020191C00F021F9031C8A
S11386B0181C00F04DFEC046941B002080B582B00B
S11386C000AF7860FEE7C04680B584B000AF786044
S11386D0FCF71AF9031CFB60FEF79CFC031CBB604F
S11386E0114B00221A70114B00221A701049BA68FB
S11386F0104B081C111C1A1CFEF7D0FB0B49BA685E
S11387000C4B081C6021FEF78FFCBB68181CFCF79F
S113871003F90549FA68074B081C6021FEF784FC3D
S11387200A20F7F7DBFFE9E7981B0020F81B00207D
S1138730AC9E00002CA2000080B584B004AF0C49AC
S11387400C4AE1235B0001200090002001900020EE
S1138750029000200390081C111C1A1C0023F7F738
S113876007FF031C012B00D0FEE7BD4680BDC046B9
S1138770C9860000B49E000080B584B000AF3A60A2
S11387801A1CFB1D1870BB1D19707B1D1A70FB1D74
S11387901B78552B1ED1BB6901221A703B1C0F3369
S11387A03A6812781A703B1C0F331B78012B05D1E1
S11387B00B4B1B6A181CFFF79BF809E03B1C0F339B
S11387C01B78022B04D1064B5B6A181CFEF780FF52
S11387D0002301E0C0460023181CBD4604B080BD40
S11387E0A419002080B582B000AFF8F76BF8031C21
S11387F07B607B68632B07D87B686422D31A7B6019
S11388007B68181CF7F76AFFFCF766FBBD4602B0ED
S113881080BDC04680B500AF0C4B1B78012B07D040
S1138820022B0BD0002B0CD1084B01221A70F3E75A
S1138830FFF7D8FF054B02221A7003E0FCF744FB54
S113884000E0C046C046BD4680BDC046581C00205E
S113885080B500AFFF20FDF7ADFA031C002B03D059
S1138860024B181C00F0A8F8BD4680BDBC9E000059
S113887080B582B000AF7860FFF7EAFF044B0022B6
S11388801A70FFF7C7FF0520F7F728FFF9E7C0467E
S1138890581C002080B584B004AFFCF70FFB104BCC
S11388A0181CFDF779FA031C002B03D00D4B181C80
S11388B000F082F80C4A0D4B032100910021019134
S11388C00021029100210391101C191CC8220023CD
S11388D0F7F74EFE031C012B00D0FEE7BD4680BD1A
S11388E040A20000E09E000071880000089F000084
S11388F080B500AFFEF77AF800F006FDF7F720FF29
S1138900FEE7C04680B500AFBD4680BD80B582B0ED
S113891000AF021CFB1D1A70FB1D1B78181C00F015
S1138920CBF8BD4602B080BD80B582B000AF021C5A
S1138930FB1D1A70FB1D1B78181C00F009F9BD46BD
S113894002B080BD80B582B000AF021CFB1D1A705E
S1138950FB1D1B78181C00F0F1F8BD4602B080BD69
S113896080B582B000AF021CFB1D1A70FB1D1B7882
S1138970181C00F0F7F8BD4602B080BD80B582B087
S113898000AF7860396072B6FEE7C04680B500AFCC
S1138990FAF7AAFABD4680BD80B500AFBD4680BDDA
S11389A080B500AF72B6FEE780B500AFBD4680BDAE
S11389B080B500AFBD4680BD80B582B000AF7860A1
S11389C0FEF728FB031C5B687A68101C191CFEF771
S11389D0A5F8BD4602B080BD80B584B000AF021CCE
S11389E0BB1D1A80BB1D1B881B0A9BB21A1CFF23CC
S11389F013407F3BFB60FB681A1C803203DA802340
S1138A005B42FB6004E0FB687F2B01DD7F23FB609E
S1138A10FB68DBB25BB2181CBD4604B080BDC04627
S1138A2090B587B000AFF860B9607A603B603C1CD9
S1138A3017340120FFF764FD031C23703B1C17331C
S1138A401B78002B03D03B1C17331B7830E03C1CF5
S1138A5017343B1C1033181CFFF776FD031C2370DE
S1138A603B1C17331B78002B03D03B1C17331B789C
S1138A701EE03B1C10331A88FB681A803B1C103321
S1138A805A88BB681A803B1C10331B88181CFFF7DC
S1138A90A3FF031C1A1C7B681A703B1C10335B88F1
S1138AA0181CFFF799FF031C1A1C3B681A7000235B
S1138AB0181CBD4607B090BD80B582B000AF021C43
S1138AC0FB1D1A70FB1D1A780123134002D00020ED
S1138AD0FDF728FEFB1D1A780223134002D0012063
S1138AE0FDF720FEFB1D1A780423134002D0022058
S1138AF0FDF718FEFB1D1A780823134002D003204B
S1138B00FDF710FEFB1D1A781023134002D0042039
S1138B10FDF708FEFB1D1A782023134002D0052020
S1138B20FDF700FEFB1D1A784023134002D00620F7
S1138B30FDF7F8FDBD4602B080BDC04680B582B0E9
S1138B4000AF021CFB1D1A70BD4602B080BDC046BA
S1138B5080B582B000AF021CFB1D1A70BD4602B086
S1138B6080BDC04680B586B002AF021CFB1D1A70E2
S1138B70FB1D1B78062B00D9BCE09A005F4BD31871
S1138B801B689F46FEF746FA031C5B685C4A101C90
S1138B90191CFDF7C3FF3B1C0F3341221A703B1C09
S1138BA00F3300220092181C01215422FF23FDF7E9
S1138BB00FF8A0E0FEF72EFA031C5B68514A101C64
S1138BC0191CFDF7ABFF3B1C0F3342221A703B1CF0
S1138BD00F3300220092181C01215422FF23FCF7BA
S1138BE0F7FF88E0FEF716FA031C5B68464A101C80
S1138BF0191CFDF793FF3B1C0F3343221A703B1CD7
S1138C000F3300220092181C01215422FF23FCF789
S1138C10DFFF70E0FEF7FEF9031C5B683B4A101CA3
S1138C20191CFDF77BFF3B1C0F3344221A703B1CBD
S1138C300F3300220092181C01215422FF23FCF759
S1138C40C7FF58E0FEF7E6F9031C5B68304A101CC6
S1138C50191CFDF763FF2F4B1B785A425341DBB2BB
S1138C601A1C2C4B1A703B1C0F3345221A703B1CE8
S1138C700F3300220092181C01215422FF23FCF719
S1138C80A7FF38E0FEF7C6F9031C5B68224A101CF4
S1138C90191CFDF743FF214B1B785A425341DBB2A9
S1138CA01A1C1E4B1A703B1C0F3346221A703B1CB5
S1138CB00F3300220092181C01215422FF23FCF7D9
S1138CC087FF18E0FEF7A6F9031C5B68144A101C22
S1138CD0191CFDF723FF3B1C0F334B221A703B1C5E
S1138CE00F3300220092181C01215422FF23FCF7A9
S1138CF06FFF00E0C046BD4604B080BD4CA200003A
S1138D00109F0000209F0000309F0000409F000043
S1138D10509F000014F0FF1F609F0000591C0020AA
S1138D20709F000090B595B000AF7860B84B5B6859
S1138D30181CFEF777FC031C002B01D1012400E072
S1138D400024B34B9B68181CFEF72EFC031C002B5D
S1138D5001D1022300E00023221C1343DCB2AC4BFC
S1138D60DB68181CFEF7E0FB031C002B01D1042375
S1138D7000E00023221C1343DCB2A54B1B69181C22
S1138D80FEF794FB031C002B01D1082300E0002311
S1138D90221C1343DCB29E4B5B69181CFEF752FD88
S1138DA0031C002B01D1102300E00023221C1343D9
S1138DB0DCB2974B9B69181CFEF704FD031C002BC7
S1138DC001D1202300E00023221C1343DCB2904B8A
S1138DD0DB69181CFEF7B6FC031C002B01D14023F1
S1138DE000E00023221C1343DAB23B1C4F331A70F9
S1138DF03B1C083300221A703B1C4F331A780123A2
S1138E00134001D0834B00E0834B3A1C0832101C02
S1138E1040211A1CF9F7DCFA3B1C4F331A78022361
S1138E20134001D07D4B00E07D4B3A1C0832101CEE
S1138E3040211A1CF9F7CCFA3B1C4F331A7804234F
S1138E40134001D0774B00E0774B3A1C0832101CDA
S1138E5040211A1CF9F7BCFA3B1C4F331A7808233B
S1138E60134001D0714B00E0714B3A1C0832101CC6
S1138E7040211A1CF9F7ACFA3B1C4F331A78102323
S1138E80134001D06B4B00E06B4B3A1C0832101CB2
S1138E9040211A1CF9F79CFA3B1C4F331A78202303
S1138EA0134001D0654B00E0654B3A1C0832101C9E
S1138EB040211A1CF9F78CFA3B1C4F331A784023D3
S1138EC0134001D05F4B00E05F4B3A1C0832101C8A
S1138ED040211A1CF9F77CFA7B685B685B493A1CF1
S1138EE00832081C111C1A1CFEF76EF9381C4C3091
S1138EF0391C4A313A1C49323B1C4833FFF790FD78
S1138F00031C002B52D13A1C0832514B101C402137
S1138F101A1CF9F739FA3B1C4C331B883A1C0832EB
S1138F20101C40211A1CF9F7EDFC3A1C0832494B7D
S1138F30101C40211A1CF9F74BFA3B1C49331B78CF
S1138F403A1C08325BB2101C40211A1CF9F75AFC77
S1138F503A1C0832404B101C40211A1CF9F738FA0D
S1138F603B1C4A331B883A1C0832101C40211A1C33
S1138F70F9F7C8FC3A1C0832364B101C40211A1C65
S1138F80F9F726FA3B1C48331B783A1C08325BB2CB
S1138F90101C40211A1CF9F735FC3A1C08322F4BDF
S1138FA0101C40211A1CF9F713FA07E03A1C083286
S1138FB02B4B101C40211A1CF9F7E6F97B685B68FF
S1138FC028493A1C0832081C111C1A1CFEF7FCF82C
S1138FD0254B1B78002B01D0244B00E0244B7A68EE
S1138FE052682449081C191CFEF7EEF8224B1B7822
S1138FF0002B01D0214B00E0214B7A6852681349C1
S1139000081C191CFEF7E0F8BD4615B090BDC0461B
S1139010A4190020809F0000889F0000909F0000FA
S1139020989F0000A09F0000A89F0000B09F000030
S1139030B89F0000C09F0000C89F0000D09F0000A0
S1139040D89F0000E09F0000EC9F0000F89F000004
S113905004A000000CA0000010A0000018A0000054
S11390601CA0000030A00000591C00203CA00000FF
S113907054A000006CA0000014F0FF1F78A00000B2
S113908090A0000080B584B000AFF860B9607A6049
S1139090FA68284B101C191C00F085F9031C002BDE
S11390A008D0FA68244B101C191C00F07CF9031C2E
S11390B0002B16D17B685B682049214A081C111CCF
S11390C01A1CFEF76DF87B685B681E491E4A081C73
S11390D0111C1A1CFEF764F8BB6801221A700023E5
S11390E024E0FA68194B101C191C00F05CF9031CED
S11390F0002B08D0FA68164B101C191C00F053F909
S1139100031C002B11D17B685B680C49114A081CB5
S1139110111C1A1CFEF758F87B68181CFFF702FE96
S1139120BB6801221A70002300E00023181CBD460E
S113913004B080BDA8A00000B0A00000BCA0000046
S1139140C0A00000D8A00000E8A000000CA100000E
S113915014A1000020A1000080B58EB002AF786099
S1139160FDF758FF031C5B68604A101C191CFDF7CF
S1139170D5FC5F4B181CF7F7B1FA3B1C2E330022C9
S11391801A803B1C2D337F221A703B1C2C337F2208
S11391901A70381C2A30391C28313A1C27323B1CDF
S11391A02633FFF73DFC031C002B09D0FDF732FFEB
S11391B0031C9B684F4A101C191CFDF7AFFC76E09A
S11391C04D4B1B78002B72D03B1C27331B783A1C69
S11391D02D32127852B25BB29A4209D13B1C26332B
S11391E01B783A1C2C32127852B25BB29A425ED08F
S11391F03A1C0C32414B101C18211A1CF9F7C4F804
S11392003B1C27331B783A1C0C325BB2101C182110
S11392101A1CF9F7F7FA3B1C0C33181C18212C22E2
S1139220F9F708F93B1C26331B783A1C0C325BB265
S1139230101C18211A1CF9F7E5FA3A1C0C32304BB1
S1139240101C18211A1CF9F7C3F8FDF7E3FE031CE0
S11392505B683A1C0C32101C191CFDF75FFC264B92
S11392601B78002B17D03B1C27331B78DAB23B1C2E
S113927024331A703B1C26331B78DAB23B1C24338C
S11392805A703B1C243300220092181C02215322E2
S1139290FF23FCF79DFC3B1C2D333A1C273212782C
S11392A01A703B1C2C333A1C263212781A703B1C61
S11392B02E331A88FA235B009A4208D9114B1B6A91
S11392C0181CFEF715FB3B1C2E3300221A80FDF7F9
S11392D0EFF8FDF773FA6420F7F700FA3B1C2E331E
S11392E03A1C2E32128864321A8052E724A10000FC
S11392F0B80B000044A10000591C00205CA1000030
S113930020A10000A419002080B584B004AFFFF7A9
S113931013FAFFF7BFFA0C4A0C4B0221009100210B
S113932001910021029100210391101C191CC822F3
S11393300023F7F71DF9031C012B00D0FEE7F7F714
S1139340FFF9BD4680BDC0465991000064A10000EC
S113935038B5051C00F00AF900F0B0F8084C236891
S1139360002B02D0984700202060064C2168002979
S113937002D0884700222260281CFFF79FF938BDDD
S11393805C1C0020601C002010B50023934203D015
S1139390CC5CC4540133F9E710BD10B5041C00F0D3
S11393A029F8201C10BD00B503780A78934204D133
S11393B0002B04D001300131F6E7981A00E0181CA4
S11393C000BD00B5431E01331A78002AFBD1181AD8
S11393D000BD30B5002393420AD0C45CCD5CAC42DE
S11393E001D0601B05E00133002CF4D1201C00E007
S11393F0002030BD30B5C9B2031C1F2A31D9444204
S11394000323234005D0D21AC51801700130A842A5
S1139410FBD1002905D00D060C042C430B0221437B
S113942019435409031C002C0ED0251C013D19605E
S113943059609960D960196159619961D961203382
S1139440002DF3D16301C318D006400F07D0041CCC
S11394501D1C013C02C5002CFBD180001B180324F9
S113946022409D18002A03D019700133AB42FBD16E
S113947030BD000010B50B4C0B4B9C4202D001CC0C
S11394808047F9E7094C0A48844202D008CC98473F
S1139490F9E7084C08498C4202D004CC9047F9E71C
S11394A010BDC04668A2000068A2000068A20000C7
S11394B068A2000068A2000068A2000010B5084C71
S11394C0084B9C4202D004CC9047F9E7064C07486D
S11394D0844203D0043C21688847F8E710BDC046A5
S11394E068A2000068A2000068A2000068A2000050
S11394F000B588421FD0002A1DD00323194207D18A
S1139500184205D19A4203D908C9043A08C0F2E7BF
S11395100123194209D1184207D19A4205D90B886F
S1139520023A038002310230E5E70B78013A037016
S113953001310130DFE700BD38B50B4D002D11D0EE
S113954000242B191968002906D02B1958689A6829
S1139550FFF7CEFF0C34F4E75A68002AF5D1986877
S11395600028F2D138BDC04680A20000054B10B5DA
S11395701C68002C04D0A068616888472468F8E758
S113958010BDC046701C0020054B181C002805D0D7
S1139590854681B00020C043009001B0F746704773
S11395A000300020F7467047F0C041464A46534613
S11395B00EC05946016071464160694681600020D1
S11395C07047704749444C450000000009090000F9
S11395D00D0A00002D333237363800002D32313475
S11395E03734383336343800000000004552523ADC
S11395F0205278207175657565206F766572666C8A
S11396006F77210D0A0000004552523A205278200B
S113961051756575652066756C6C3F0D0A00000018
S11396204552523A2052657472790D0A00000000C6
S11396304552523A205265747279206661696C65AC
S113964064210D0A000000004552523A2054696D0D
S1139650656F75740D0A0000494E495449414C0028
S1139660414C574159535F4F4E0000005452414EF4
S1139670534D49545F4441544100000057414954FB
S1139680494E475F444154415F53454E54000000E6
S113969052454144595F54585F525800434845432A
S11396A04B5F545800000000504F5745525F444FE1
S11396B0574E0000554E4B4E4F574E007261646931
S11396C06F00000047726F7570206F6620726164CE
S11396D0696F20636F6D6D616E64730D0A00000025
S11396E0202068656C707C7374617475730000006D
S11396F053686F777320726164696F2068656C705A
S1139700206F72207374617475730D0A0000000079
S113971020206368616E6E656C203C6E756D6265B9
S1139720723E0000537769746368657320746F2018
S113973074686520676976656E206368616E6E651E
S11397406C2E204368616E6E656C206D7573742099
S1139750626520696E207468652072616E67652099
S1139760302E2E3132370D0A000000002020706F99
S1139770776572203C6E756D6265723E0000000074
S11397804368616E676573206F75747075742070BB
S11397906F77657220746F20302C202D31302C208F
S11397A02D31322C202D31380D0A00002020736E0B
S11397B0696666206F6E7C6F666600005475726E13
S11397C07320736E696666696E67206F6E206F72B0
S11397D0206F66660D0A0000202077726974657236
S11397E0656720307852656720307856616C0000D8
S11397F057726974652061207472616E7363656960
S11398007665722072656769737465720D0A00006B
S11398102020666C75736800456D70747920616CE6
S11398206C207175657565730D0A000020207072D7
S1139830696E7472656700005072696E7420746892
S11398406520726164696F207265676973746572FB
S1139850730D0A00202061646472203078000000D7
S11398600D0A0000526164696F00000020207374C7
S1139870617465007965730D0A0000006E6F0D0A4E
S1139880000000002020736E696666002020636873
S1139890616E6E656C0000002064426D0D0A00006C
S11398A02020706F77657200206B6270730D0A0060
S11398B02020646174612072617465003078000056
S11398C03A20000052585F445220000054585F442C
S11398D0532000004D41585F52542000527846698D
S11398E0666F456D70747920000000005278556EE3
S11398F07573656420000000527850233520000001
S11399005278502334200000527850233320000032
S11399105278502332200000527850233120000026
S1139920527850233020000054585F46554C4C2048
S113993000000000202053544154555300000000FF
S1139940524555534520000054585F454D505459D5
S11399502000000052585F46554C4C200000000087
S113996052585F454D50545920000000202046496C
S1139970464F5F535441545553000000206C6F739D
S1139980742C20002072657472790D0A00000000A6
S113999020204F4253455256455F54580000000062
S11399A068656C7000000000726164696F2068650E
S11399B06C70000073746174757300007261646983
S11399C06F207374617475730000000072616469C0
S11399D06F20736E696666206F6E00007261646941
S11399E06F20736E696666206F66660072616469D3
S11399F06F206368616E6E656C00000057726F6E55
S1139A006720617267756D656E742C206D75737453
S1139A1020626520696E207468652072616E6765D6
S1139A2020302E2E3132380D0A0000007261646934
S1139A306F20706F7765720057726F6E6720617266
S1139A4067756D656E742C206D7573742062652066
S1139A50302C202D31302C202D3132206F72202DCE
S1139A6031380D0A00000000726164696F2077725A
S1139A70697465726567000057726F6E6720617262
S1139A8067756D656E74730D0A0000007261646918
S1139A906F20666C75736800466C757368696E67D1
S1139AA0206661696C6564210D0A00007261646955
S1139AB06F207072696E747265670000726E776BE6
S1139AC00000000047726F7570206F6620726E7719
S1139AD06B20636F6D6D616E64730D0A000000008E
S1139AE0202068656C707C73746174757300000069
S1139AF053686F77732068656C70206F722073747D
S1139B00617475730D0A00000D0A000030780000BE
S1139B10202061646472000068656C7000000000BD
S1139B20726E776B2068656C7000000073746174EA
S1139B3075730000726E776B2073746174757300B3
S1139B405241434B000000004E41434B00000000D3
S1139B50444154410000000041434B00434D440044
S1139B605061636B65742054782000005061636B0E
S1139B706574205278200000666C6167733A200097
S1139B802800000049535F41434B2C005245515F6C
S1139B9041434B00290000002073697A653A200094
S1139BA02050485920646174613A2000200000006C
S1139BB0204D41432073697A653A0000207479701E
S1139BC0653A00002073233A00000000204E574BF2
S1139BD0207372633A000000206473743A0000003A
S1139BE02041505020747970653A00002073697ADE
S1139BF0653A00000D0A00004652544F53310000EC
S1139C000D0A00005441534B204C4953543A0D0A59
S1139C104E616D65090953746174757309507269F5
S1139C206F09537461636B09544342230D0A0000A6
S1139C302D2D2D2D2D2D2D2D2D2D2D2D2D2D2D2D50
S1139C402D2D2D2D2D2D2D2D2D2D2D2D2D2D2D2D40
S1139C502D2D2D2D2D2D2D2D2D2D2D2D2D2D2D2D30
S1139C602D2D2D2D2D2D2D2D2D2D2D2D2D2D00007A
S1139C700D0A2A2A2A206F7574206F662068656190
S1139C807021202A2A2A0D0A0000000020205254A4
S1139C904F53207469636B730000000000000000E0
S1139CA020487A2C20000000206D730D0A0000006B
S1139CB020204672656520686561700020627974B1
S1139CC065730D0A0000000047726F7570206F669F
S1139CD0204652544F533120636F6D6D616E64732F
S1139CE00D0A0000202068656C707C7374617475C3
S1139CF0730000005072696E742068656C70206F88
S1139D00722073746174757320696E666F726D610D
S1139D1074696F6E0D0A000068656C7000000000C5
S1139D204652544F53312068656C700073746174EB
S1139D30757300004652544F533120737461747527
S1139D407300000068656C7000000000434C5331E0
S1139D502068656C700000000D0A00002D2D2D2D6B
S1139D602D2D2D2D2D2D2D2D2D2D2D2D2D2D2D2D1F
S1139D702D2D2D2D2D2D2D2D2D2D2D2D2D2D2D2D0F
S1139D802D2D2D2D2D2D2D2D2D2D2D2D2D2D2D2DFF
S1139D902D2D2D2D2D2D2D2D2D2D00004A6F797358
S1139DA07469636B00000000434C533100000000F1
S1139DB047726F7570206F6620434C533120636F78
S1139DC06D6D616E64730D0A0000000020206865EB
S1139DD06C707C7374617475730000005072696EEA
S1139DE0742068656C70206F72207374617475736D
S1139DF020696E666F726D6174696F6E0D0A000082
S1139E007374617475730000434C5331207374612F
S1139E1074757300434D443E200000000D0A5359ED
S1139E205354454D205354415455530D0A000000DA
S1139E304669726D77617265000000004A756E2094
S1139E4031372032303134002000000031333A33CE
S1139E50363A3236000000002A2A2A204661696C0C
S1139E606564206F7220756E6B6E6F776E20636F02
S1139E706D6D616E643A20002A2A2A205479706537
S1139E802000000020746F206765742061206C69D5
S1139E907374206F6620617661696C61626C652001
S1139EA0636F6D6D616E64730D0A000068656C709C
S1139EB0000000005368656C6C0000004552523A83
S1139EC0204661696C65642073657474696E6720EB
S1139ED06E6F646520616464726573730D0A0000BB
S1139EE04552523A206661696C65642073657474E6
S1139EF0696E67206D6573736167652068616E6460
S1139F006C6572210D0A0000524E65740000000059
S1139F10412070726573736564210D0A00000000AE
S1139F20422070726573736564210D0A000000009D
S1139F30432070726573736564210D0A000000008C
S1139F40442070726573736564210D0A000000007B
S1139F50452070726573736564210D0A000000006A
S1139F60462070726573736564210D0A0000000059
S1139F704B45592070726573736564210D0A0000A6
S1139F8041284F4E2920000041286F666629200091
S1139F9042284F4E2920000042286F66662920007F
S1139FA043284F4E2920000043286F66662920006D
S1139FB044284F4E2920000044286F66662920005B
S1139FC045284F4E2920000045286F666629200049
S1139FD046284F4E2920000046286F666629200037
S1139FE04B4559284F4E290D0A0000004B4559286E
S1139FF06F6666290D0A00002020427574746F6E26
S113A00073000000583A2030780000002800000057
S113A0102920593A20307800290D0A0047657458E0
S113A020592829206661696C6564210D0A000000C5
S113A0302020416E616C6F67000000007965732019
S113A04028746F67676C6520776974682046290DEA
S113A0500A0000006E6F2028746F67676C652077B4
S113A0606974682046290D0A0000000020204A6F08
S113A07079737469636B00007965732028746F6762
S113A080676C6520776974682045290D0A00000013
S113A0906E6F2028746F67676C6520776974682019
S113A0A045290D0A0000000068656C70000000007E
S113A0B06170702068656C70000000006170700051
S113A0C047726F7570206F662061707020636F6DCA
S113A0D06D616E64730D0A00202068656C707C737A
S113A0E074617475730000007072696E7420686521
S113A0F06C70206F722073746174757320696E665E
S113A1006F726D6174696F6E0D0A0000737461740F
S113A110757300006170702073746174757300004E
S113A1200D0A000048656C6C6F2066726F6D2074B8
S113A1306865204A6F79737469636B20417070217C
S113A1400D0A00004661696C656420746F206765C0
S113A1507420782F79210D0A0000000078793A20C4
S113A1600000000041707000080000001122334418
S113A170550000000A3800001638000016390000A7
S113A1808A380000C83800002A3800005838000017
S113A190163900006A3A00006E3A0000723A000074
S113A1A0763A0000863A00007A3A00007E3A0000CF
S113A1B0823A00009A440000B0440000C644000003
S113A1C0DC440000F2440000084500007E45000025
S113A1D08E4500009E450000AE450000BE450000CF
S113A1E0CE4500005A46000068460000764600004E
S113A1F08446000092460000A0460000CD480000BE
S113A2005548000091480000E94800003D41000025
S113A210054E000000000000F17100003D720000D6
S113A2203D7200009972000048490000496B00002B
S113A23091660000E94E00008590000000000000D7
S113A240D54600007987000000000000848B0000E0
S113A250B48B0000E48B0000148C0000448C0000DC
S10BA260848C0000C48C000092
S113A268FFFFFFFFAAAAAAAA08270000FF00000010
S10BA27818A20000010000001F
S113A28068A2000000F0FF1F18000000000000009A
S10BA2900000000000000000C2
S903868DE9
